:020000040800F2
:104000000050002035D50008A5A60008A7A6000886
:10401000A9A60008ABA60008ADA600080000000095
:10402000000000000000000000000000B1A6000831
:10403000AFA6000800000000B3A60008297E000813
:10404000B5A60008B7A60008B9A60008BBA60008D8
:10405000BDA60008BFA60008C1A60008C3A60008A8
:10406000C5A60008C7A60008C9A6000800000000F1
:104070000000000000000000000000000000000040
:104080000000000000000000D9A60008DBA6000820
:10409000E9A60008F9A6000809A7000819A7000862
:1040A0001BA700081DA700081FA7000821A70008DC
:1040B000FD94000825A7000827A7000829A70008E5
:1040C0008DA200082DA7000811A30008D9930008AD
:1040D00033A700083976000837A7000839A7000879
:1040E0003BA700083DA700083FA70008000000000C
:1040F00000000000000000000000000000000000C0
:0C41000000000000000000005FF800005C
:1041100030BF704720BF704740BF7047BFF36F8FFD
:104120007047BFF34F8F7047BFF35F8F704701DF5A
:104130007047EFF31480704780F31488BFF36F8FDC
:104140007047EFF30980704780F309887047EFF3F9
:104150000880704780F30888704772B6704762B66F
:10416000704771B6704761B6704780F31188704729
:10417000EFF31280704740BA704700BA70470000F2
:104180002DE9F7434B4D4C48012107F0F7FB042084
:10419000012108F0BFF80324102742F21813284623
:1041A00001A94FF00408ADF804308DF806404FF037
:1041B00018098DF8077007F052FB4FF480733F4EDB
:1041C000C5F8109028466B610DEB080144F2060318
:1041D000ADF804308DF806408DF8078007F03FFBFE
:1041E0000820012108F096F841F2180330460DEB43
:1041F0000801ADF804308DF806408DF8077007F01F
:104200002EFB4FF48053C6F81490304633610DEB0B
:10421000080144F22443ADF804308DF806408DF8CF
:10422000078007F01CFB4FF400633046ADF8043004
:104230000DEB080148238DF807308DF8064007F094
:104240000EFB3846012108F065F88DF806401C4C3D
:104250004FF4004620460DEB0801ADF804608DF8E0
:10426000077007F0FCFA01212661164807F086FB6B
:1042700000230A211A464FF400506861AC68286197
:10428000A868640458BF0132400448BF01330139B3
:10429000F1D10A2A0C4A03D10A2B01D1012300E0F3
:1042A000002305480121137007F068FB03B0BDE847
:1042B000F08300BF0008014000023000000C014004
:1042C00000100140000430002C2D0020104B82B063
:1042D0001B78D3B10F4B4FF400425A610022019278
:1042E000019945F2CD62914202D8019A0132F6E776
:1042F0004FF400421A6100230193019A45F2CD6305
:104300009A42E7D8019B0133F6E702B0704700BF3D
:104310002C2D00200010014010B1012802D0704760
:10432000102200E00822014B5A617047000C014046
:1043300010B1012802D07047102200E00822014B82
:104340001A617047000C014038B50546002445FA53
:1043500004F3DB07E0B202D5FFF7EAFF01E0FFF765
:10436000DBFF0134082CF2D138BD08B5032818D87A
:10437000DFE800F00204090E0B4B05E00A4B9868D9
:10438000C0F3400008BD094B9868C0F3800008BD29
:10439000002003F023FEB0F5006F94BF0020012041
:1043A00008BD002008BD00BF00080140000C01400E
:1043B00030B1012809D1064BD868C0F3C00070475E
:1043C000034BD868C0F3001070470020704700BF4F
:1043D000000C014038B500242546E0B2FFF7C5FFC8
:1043E00018B10123A3401D43EDB20134082CF4D1D0
:1043F000284638BD20B9034B9868C0F38020704729
:1044000000207047000C014010B9C90804F042BAFE
:10441000704708B107F0BCBD07F0C2BD62B6704777
:1044200072B6704710B9024B08225A61704700BF3C
:104430000008014010B9024B08221A61704700BF02
:10444000000801407047074B9A88C2F30722032AED
:1044500006D19A88D2B2FD2A02D1188980B270475B
:1044600000207047006C0040194B70B59D68194CD6
:1044700015F4006529D1FF212A46284600F040FAAC
:1044800001220646FF21284600F03AFA40EA0620BB
:1044900010F002034FEA900018BF0123C2042370FA
:1044A00003D5237843F002032370830403D52378D4
:1044B00043F004032370084A636892F828201840E8
:1044C000A06012B1034A181A9060A06870BD00BFC6
:1044D000000C01408004002008000020F8B5604B6B
:1044E0009B681B0500F1BA8003F0F0FC5D4DE860AD
:1044F000FFF7BAFF6C692861A042294634DD8B6959
:10450000051B9D42584B0CDA1C68D1E908236C430B
:10451000121943EBE473C1E908238B6A1D448D62D1
:1045200059E091F82C6077070CD54C681A68041B89
:10453000624326F00406D317C1E908238C6281F890
:104540002C6033E04E681B68241A344404FB0334A7
:10455000D1E90823121B63EBE473C1E90823F64396
:104560008B6A35442B4411E035DAAB69221A9A4242
:104570003D4B0DDA1D68041B5543D1E90823521B3E
:1045800063EBE573C1E908238B6A23448B6222E065
:1045900095F82C506A070ED51A6825F00405424399
:1045A000D317C1E90823886281F82C500022002328
:1045B000C1E90C230FE04A681D680132041B144452
:1045C0006543D1E90823521943EBE573C1E9082398
:1045D0008B6A1C448C628C6A8E6BCA6BA61B86EA43
:1045E000E675A5EBE67595421E4B2CD942F210728A
:1045F0005643DF681D6C3C227D1B5D6496FBF5F520
:104600006A431F645F689C63013792FBF7F29A6408
:1046100040F6B834002AB8BF5242A24201DDC82297
:1046200003E0B2F57A7F02DD6422DA6315E0322A14
:1046300001DD0A22F9E70A2A01DD0522F5E7012A50
:104640000BDD0122F1E7DC681A6CA21AB2F5FA6FF1
:1046500003D90122DA6300229A644861F8BD00BFE1
:10466000000C0140800400200400002008B568B957
:10467000FFF734FF0649D1E90823D1E90C01121AEA
:1046800063EB0103100A40EA036008BD002008BD87
:104690008004002038B50D46F8B9104CFFF71EFF16
:1046A000D4E908016268002871F100034FEA022290
:1046B00002DA404261EB4101D31709F033FDC4E94E
:1046C0000C23E9170B022A02D4E90C0143EA156313
:1046D000121843EB0103C4E9082338BD800400200D
:1046E00010B9024B09011960704700BF0400002097
:1046F00010B9024B83F82C10704700BF80040020D3
:10470000014B986C704700BF8004002010B9024B29
:1047100018787047002070478004002038B5214B7E
:10472000214A1B69002059090901204C03F01F038D
:104730001160FE21024684F82C3000F0E1F840219F
:104740000122002000F0DCF800200146024600F0C3
:10475000D7F8054600200146012200F0D1F8082DC7
:1047600005D140F6FF7363604FF4006304E040F24C
:10477000FF3363604FF400730020E7210246A3611A
:1047800000F0BEF800200146012200F0B9F8FFF762
:104790006BFE60610002C117C4E90C01C4E90801A5
:1047A00038BD00BF342D002004000020800400200C
:1047B00008B5FFF759FE052808D9FFF755FE40F266
:1047C000F933984294BF0020012008BD012008BDA4
:1047D0002DE9F04F4FF4804087B0012107F0A6FD8E
:1047E0000120014607F096FD03264FF420434FF0C9
:1047F000180B69463E484FF0040AADF800308DF8BA
:1048000002608DF803B007F02AF84FF48043694640
:1048100037480024ADF8003001254FF482794FF479
:10482000007808278DF802608DF803A007F017F8CC
:104830000DEB0A012F48ADF80440ADF80690ADF835
:104840000840ADF80A40ADF80C50ADF80E80ADF858
:104850001070ADF81240ADF8144007F013FE294671
:10486000244807F095FE29464FF4805007F052FD8A
:104870002846214607F082F8A02369461E48ADF875
:1048800000308DF802608DF803B006F0E8FF69464D
:1048900040231948ADF800308DF802608DF803A070
:1048A00006F0DDFF0223ADF80A30ADF80440ADF8A4
:1048B0000690ADF80840ADF80C50ADF80E80FFF74B
:1048C000C2FD484528BF102301A90C482CBFADF8F4
:1048D0001030ADF81070ADF81240ADF8144007F08C
:1048E000D1FD0648012107F053FE07B0BDE8F08F67
:1048F000000C014000380040000801400030014039
:1049000038B50D461446E8B90F4B4FF480525A6142
:104910000E48022107F0C0FE0028F9D00B482946B6
:1049200007F066FE0948012107F0B6FE0028F9D01D
:104930001CB1054B4FF480521A61044807F05AFE2F
:10494000C0B238BD002038BD000C01400038004026
:1049500038B5CE4DA8786B7808B1042254E2AA2B62
:1049600000F0F28175D8822B00F0518134D8052BEC
:1049700000F0248116D8022B00F0F9800BD8002B10
:1049800000F0EF80012B40F03E82D5F80300BDE837
:10499000384004F049BF032B00F0F680042B00F0F0
:1049A000008130E20C2B00F0198109D8062B00F0B1
:1049B0000F81072B40F02782EA78B54B9A720AE103
:1049C0000D2B00F01881802B40F01D82D5F80300DC
:1049D000BDE8384004F042BFA42B00F070811FD81E
:1049E000A12B00F05D810DD88C2B00F01A81A02B3B
:1049F00040F00982D5F803100020C9B2BDE8384064
:104A000003F0F8BDA22B00F05281A32B40F0FB81F4
:104A1000D5F803100020C9B2BDE8384003F020BE2D
:104A2000A72B00F0828106D8A52B00F05A81A62B77
:104A300000F06981E7E1A82B00F07E81A92B40F00E
:104A4000E281D5F803100020C9B2BDE8384003F078
:104A5000BBBEB72B00F0BB8142D8B02B00F09281D7
:104A600025D8AD2B00F07F8113D8AB2B00F07381DC
:104A7000AC2B40F0C881D5F803100020C9B203F078
:104A8000C1FEAA78834B03EBC203D5F803205A7109
:104A900038BDAE2B00F06E81AF2B40F0B481D5F85D
:104AA00003100020C9B2BDE8384003F019BFB32B92
:104AB00000F077810DD8B12B00F06B81B22B40F064
:104AC000A281D5F803100020C9B2BDE8384003F038
:104AD00025BFB52B00F06C81B62B00F06E8192E102
:104AE000CC2B00F0B78019D8C22B00F0A1800AD8D7
:104AF000B82B00F07981C12B40F08581D5F80320D7
:104B0000634B1A7238BDC32B00F09B80C82B40F05A
:104B10007A81D5F803205E4BDA7738BDD42B00F0CC
:104B20009E8017D8D12B00F06781D22B40F06B818B
:104B3000D5F80320564BE9781A61002001F01F01D7
:104B4000FFF7D6FDD5F80310A8784911BDE8384025
:104B5000FFF7C6BDD62B00F08780FE2B00F08980C2
:104B600051E1D5F80300BDE8384004F057BED5F850
:104B70000300494A00F18053013B93423FF6EDAEFA
:104B8000BDE8384004F030BED5F80300424A00F1D9
:104B90008053013B93423FF6E0AEBDE8384004F05D
:104BA0002BBED5F803003C4A00F18053013B9342F1
:104BB0003FF6D3AEBDE8384004F046BED5F803005A
:104BC000B0F1007FBFF4C9AEBDE8384004F032BE9A
:104BD000EA782F4B5A720122304B16E1D5F80320A8
:104BE0002B4B1AB95A7B42F0020202E05A7B22F0A8
:104BF00002025A7338BDD5F80320254B1AB95A7BE7
:104C000042F00102F5E75A7B22F00102F1E7D5F804
:104C10000300B0F1805F3FF6A0AEBDE8384004F07D
:104C2000F3BDE8781A4BD872BDE8384004F0E0BE16
:104C3000D5F80330B3F1805F3FF68FAE144A1360AE
:104C400038BDD5F80330B3F1805F3FF686AE104A29
:104C5000536038BDD5F803200D4BDA8138BDD5F847
:104C600003200B4B5A6138BDD5F80320084B9A83BB
:104C700038BDD5F80330052B3FF66FAE034BD8781F
:104C8000034B1873BDE8384004F08ABE8828002022
:104C9000342D0020142D0020FEFFFF1F942D002036
:104CA000D5F80310BDE83840C9B203F0AFBCD5F861
:104CB00003100020C9B2BDE8384003F0C7BC03F0C0
:104CC00031FDAB78D5F8031028B91846C9B2BDE854
:104CD000384003F0D9BC1846C9B2BDE8384003F0EB
:104CE000FBBC002003F01EFDD5F8031028B9A878FE
:104CF000C9B2BDE8384003F0D1BCA878C9B2BDE85C
:104D0000384003F0FDBC002003F00CFDD5F8031083
:104D100028B9A878C9B2BDE8384003F0C9BCA87862
:104D2000C9B2BDE8384003F0E1BCD5F80310BDE8D6
:104D30003840C9B203F0C6BCD5F803100020C9B290
:104D4000BDE8384003F036BDD5F80310BDE8384063
:104D5000C9B203F043BDD5F803100020C9B2BDE8C5
:104D6000384003F045BDD5F80310BDE83840C9B25E
:104D700003F07CBDD5F80310002049B2BDE83840EF
:104D800003F07EBDD5F80310BDE83840C9B203F08A
:104D9000B1BDD5F803100020C9B2BDE8384003F01A
:104DA000B3BDD5F80310BDE83840C9B203F0CABDA1
:104DB000D5F80320164B9A6138BDD5F80300154B82
:104DC000186018BB5979BDE8384003F01BBD114B82
:104DD000D5F803201A71104B1B78012B16D1E978F6
:104DE000BDE83840FFF710BBD5F803100020C9B26A
:104DF000BDE8384003F03EBCD5F803100020BDE804
:104E00003840FFF747BC0322044B1A7038BD00BF7F
:104E1000342D0020142D0020972D0020FC28002088
:104E200038B5AF4A93781446022B00F01F81032B4C
:104E300000F02381002B40F0948153784F2B00F039
:104E4000A48037D8462B7AD014D8422B65D009D805
:104E5000402B5ED0412B40F08281D178A14B0020C5
:104E600019705EE0442B9F4A5FD064D8E17804203B
:104E7000117156E0492B72D00AD8472B67D0482BC6
:104E800040F06D81D3789749262001F8263FDAE07B
:104E90004C2B70D04D2B73D04B2B40F06081914C3C
:104EA000D1780320E17002F0D0F9E078BDE8384015
:104EB00002F058BC572B00F0B8800FD8522B7FD08F
:104EC00004D8502B68D0512B6BD048E1542B00F004
:104ED00094807CD3552B00F09C8040E1832B00F024
:104EE000B7800BD8592B00F0A6805A2B40F03781A1
:104EF000D3787C49282001F8283FA4E0852B00F0D6
:104F0000B080C0F0A980FF2B40F02981D278764B89
:104F100029E140F2FF70D17803E0D178714B012094
:104F20005970BDE8384002F090B9D4F803301C2025
:104F3000D3616E4909E0E17805205171F1E7D2F8BB
:104F4000033068490C2041F80C3F04227CE0654D99
:104F5000D2F80330294641F8083F08203EE0D278D5
:104F6000604B0AB9DA7503E061490122DA754A60DB
:104F70001720D97DD5E7D1785A4B02209970D0E718
:104F8000D178584B15205975CBE7D2F80310554B03
:104F9000C9B259761920C4E7D178524B16209975B9
:104FA000BFE7504B1A7D1D4612F0010F04D0E37885
:104FB000DB0701D402F0BAF9E17814202975B0E7D3
:104FC000D2F803304749202041F8203FBDE7454D46
:104FD000D2F80330294641F8103F1020042202F095
:104FE0004DF9444B1B78002B40F0BE806879A968CE
:104FF0002A69BDE8384002F0EFBCD2F80330012B3B
:1050000000F2AF80364B3749DB781A2001F81A3F9F
:1050100019E0D2F80330012B00F2A380304B314964
:10502000DB781B2001F81B3F0DE0D3782D492720AA
:1050300001F8273F07E0D2F803302A49242021F85D
:10504000243F022200E00122BDE8384002F016B9F8
:10505000D2F80320284B02E0D2F80320274B1A6035
:1050600038BDD2F80320244B5A6038BD5178244B08
:10507000D2F8032043F8212038BD5378282B55D08F
:1050800018D8022B49D00CD8002B3DD0012B66D16B
:105090001C4BD2F803205A6002F018FF164BD86060
:1050A00038BD092B60D0272B59D1D2F80320154BDE
:1050B000DA6038BD2B2B43D008D8292B3BD02A2BC4
:1050C0004DD1D2F803200F4B9A6138BD2D2B41D022
:1050D0003BD32E2B43D1D2F803200A4B9A6238BD22
:1050E0008828002008000020F62800202400002046
:1050F000FC280020082D0020D0040020F8280020E3
:10510000082900205C2D0020184BD2F803201A60DB
:1051100002F0DCFE164B986038BD144BD2F8032029
:105120009A6002F0D3FE124B186138BDD2F803200A
:105130000E4B1A6138BDD2F803200C4B5A6138BDB2
:10514000D2F80320094BDA6138BDD2F80320074BAF
:105150001A6238BDD2F80320044B5A6238BD0322CC
:1051600000E00422034B1A7038BD00BF5C2D002004
:10517000D0040020FC280020F7B5D14ED14F337861
:10518000D6F803006422222B7B703A707860354693
:105190003C4601F0AE815CD80F2B00F05E8627D82C
:1051A000072B00F0F48211D8032B00F0E18007D820
:1051B000012B00F0BE80022B00F0CC8001F006BC79
:1051C000052B00F0218140F2BF8021E10B2B00F084
:1051D000988506D8092B00F04C8440F29F8300F09C
:1051E0004CBC0D2B00F0C08540F2A88500F0F5BD49
:1051F000192B00F07B8714D8152B00F0CE8607D82A
:10520000132B00F06D86142B00F0A58601F0DEBB99
:10521000172BAD4B00F0508700F25B87986101F0CF
:10522000D7BB1E2B00F07E850CD81B2B00F080878F
:10523000C0F06D871C2B41F0C983A34B00221A7567
:1052400001F0C6BB202B01F0C18041F2868001F045
:10525000FCB8812B01F0E98135D8412B01F0D381D5
:1052600017D8252B01F0808107D8232B01F0488126
:10527000242B01F04C8101F0A9BB272B01F0B58153
:10528000C1F08E81402B41F0A18302F03AFF01F082
:105290009FBB452B01F0C08108D8432B01F0B6819C
:1052A00001F2B78102F02FFF01F092BB472B01F012
:1052B000B981C1F0B481802B41F08883824B0022F8
:1052C0001A7501F085BB882B01F02B821BD8842B2B
:1052D00001F0DC810DD8822B01F0BB81832B41F0E2
:1052E0007583794B002183F8401083F8281101F071
:1052F000B4B9862B01F0DB8101F24882724B0022A7
:105300001A7501F065BB8C2B01F09B8206D88A2BA5
:1053100001F07B8241F2618201F08EBAF22B01F042
:105320001B83FF2B01F049838D2B41F04F8301F04C
:10533000D0BAB37853B9012004F090FAD6F803003C
:1053400004F052FA01F044BBB378FBB1042323709C
:1053500001F03EBBB378002BF8D1012004F07EFAB7
:10536000574BD3F80300404204F03EFA01F030BB43
:10537000B578002DEAD1284604F0B2FD012004F0F2
:105380006DFA284604F030FA01F022BB4C4B5B78F2
:10539000032B35D8DFE803F00209152104F03EFAAB
:1053A000002004F05BFA01F013BB04F07FFAD6F89A
:1053B0000330184404F032FA002004F04FFA01F0F0
:1053C00007BB1428C2DC414B53F8200004F026FA36
:1053D000002004F043FA01F0FBBA1428B6DC04F014
:1053E00065FAD6F80330B2781A44384B53F82230B5
:1053F000184404F013FA002004F030FA01F0E8BA7F
:1054000003233B7001F0E4BAFFF7A2FA01F0E0BA1F
:10541000B0787378002899D1AC2B00F074816CD8E7
:10542000802B00F0008131D8062B00F0D78014D8F3
:10543000022B00F0C98008D8002B00F0C280012B9D
:1054400040F08D8104F032FAC0E0042B00F0C080FF
:1054500000F2C18004F014FAB8E00A2B00F0C78013
:1054600007D8082B00F0BD8000F2BE80184B9B7A55
:105470006FE10C2B00F0CF80C0F0C3800D2B40F00B
:105480006E81134B5B7B13F0010FC8E0A42B00F07F
:1054900006811FD8A02B00F0F78008D8822B00F0DF
:1054A000C5808C2B40F05B81094BDB7A51E1A22B4C
:1054B00000F0ED8000F2EF80002003F0BFF885E0FF
:1054C00088280020FC280020D004002094280020F8
:1054D000342D0020A82B00F00B8105D8A62B00F05E
:1054E000F78040F2E980FFE0AA2B00F0048100F28F
:1054F0000681002003F09AF968E0C32B00F09E803B
:105500002FD8B32B00F0118116D8AF2B00F00281F9
:1055100009D8AD2B00F0FA80AE2B40F0208100209E
:1055200003F0CCF952E0B12B00F0F78000F2F980E3
:10553000002003F033FA49E0B72B00F0018106D8D0
:10554000B52B00F0F78000F2F880A34BF0E0C12B00
:105550006FD071D8B82B40F00281002003F0EAF838
:1055600034E0D02B00F0888012D8C82B6BD006D83E
:10557000C42B66D0C52B40F0F280984BDEE0CE2BDA
:1055800064D065D8CC2B40F0EA80954BDB89E0E015
:10559000D62B73D00AD8D22B00F0D980C0F0D3809C
:1055A000D42B40F0DC808E4B5B69D2E0DB2B00F02B
:1055B000D280FE2B65D0D72B40F0D180FEF754FF70
:1055C00004E004F06DF901E004F052F96060C8E015
:1055D00004F07AF9FAE704F06FF9F7E7804B5B7AA9
:1055E000B7E004F099F9F1E77E4B9B6810E07E4B41
:1055F0005A7E7E4B9B680AB183F00203C3F34003DB
:10560000A7E0794B5A7E794B9B680AB183F004037B
:10561000C3F380039DE0724B5B7B13F0020F14BF5A
:105620000023012395E004F057F9CFE704F030F9A7
:10563000CCE76B4B1B7A8CE0694B7FE0684B5B6877
:1056400087E06B4B7AE0664BDB7F82E0694B75E06D
:10565000B378694A0021D05C796010B167480125B0
:105660004560D154664AD15C19B1616841F00201CC
:1056700061600021D15474E0624B59E0584B9B8B20
:1056800067E0574B1B7B64E002F0D0FF9EE70020F1
:1056900003F040F89AE7002003F044F896E703F09F
:1056A00041F8594B9B7818B9184603F04BF88DE731
:1056B000184603F067F889E7002003F033F818B9BB
:1056C000B07803F047F881E7B07803F06BF87DE736
:1056D000002003F027F818B9B07803F043F875E715
:1056E000B07803F057F871E7002003F043F86DE756
:1056F00003F092F86AE7002003F0A0F866E70020C4
:1057000003F0A4F862E7414B5B7922E0002003F04C
:10571000CBF85BE703F03AF958E7002003F046F9CD
:1057200054E7002003F04AF950E703F057F94DE73A
:105730001B780EE02A4B9B690BE0344B1B6808E09A
:10574000324B1B7905E00020FEF790FF3EE7244B2B
:105750001B69636005E00020FEF7D8FF36E70323EE
:1057600023702B4B1B78002B01F03281294B626890
:105770001A60294B2AB91A6842F008021A6001F02F
:1057800027B91A6822F008021A6001F021B9B2782C
:105790007378002A7FF4DAADB52B00F0918048D8F9
:1057A000072B00F0828009D8052B73D076D8042B04
:1057B00040F0B08004F0C2F801F00AB9822B7BD02F
:1057C0002ED80C3B012B00F2A5804D20134901225D
:1057D00001F054FD01F0FCB8122D0020582D0020DE
:1057E000342D0020000C014008000020000801407A
:1057F0000C2D0020282D00202D2D0020FC2800201D
:105800001D2D00202E2D002088280020142D002082
:10581000F7280020E828002090280020412D0020B3
:105820008C2B77D14B20C549012201F027FD01F0D7
:10583000CFB8CC2B59D016D8C22B48D008D8C12B02
:1058400068D14820BE49012201F018FD01F0C0B81E
:10585000C32B43D0C82B5DD15F20BA49012201F090
:105860000DFD01F0B5B8D42B46D008D8D22B51D1BC
:105870005020B549042201F001FD01F0A9B8D62B52
:1058800041D0FE2B46D14C20B049012201F0F6FC5C
:1058900001F09EB804F04AF801F09AB84920AC49EA
:1058A000012201F0EBFC01F093B84A20A949012242
:1058B00001F0E4FC01F08CB804F048F801F088B87D
:1058C0005820A549042201F0D9FC01F081B84020FC
:1058D000A249042201F0D2FC01F07AB84420A04988
:1058E000042201F0CBFC01F073B84E209D49022246
:1058F00001F0C4FC01F06CB854209B49042201F073
:10590000BDFC01F065B85C209849022201F0B6FCAC
:1059100001F05EB80323237001F05AB8B2787378AF
:10592000002A7FF413ADB52B75D024D8072B67D090
:1059300009D8052B59D05CD8042B40F0968004F090
:1059400015F801F045B8822B61D00AD80C3B012B29
:1059500000F28B804D208649012201F0CBFC01F042
:1059600037B88C2B40F081804B207449012201F024
:10597000C1FC01F02DB8CC2B62D016D8C22B51D06F
:1059800008D8C12B71D148206D49012201F0B2FC29
:1059900001F01EB8C32B4CD0C82B66D15F206949DB
:1059A000012201F0A7FC01F013B8D42B4FD008D886
:1059B000D22B5AD150206449042201F09BFC01F003
:1059C00007B8D62B4AD0FE2B4FD16A4C4C2004F19D
:1059D0000C01012201F08EFC674B9B7804EB431411
:1059E000207B03F0DDFF00F0F3BF03F0B7FF00F012
:1059F000EFBF49205649012201F07CFC00F0E8BFCE
:105A00004A205449012201F075FC00F0E1BF03F087
:105A1000B5FF00F0DDBF58204F49042201F06AFCB9
:105A200000F0D6BF40204D49042201F063FC00F095
:105A3000CFBF44204A49042201F05CFC00F0C8BFFB
:105A40004E204849022201F055FC00F0C1BF54200D
:105A50004549042201F04EFC00F0BABF5C204349E6
:105A6000022201F047FC00F0B3BF0323237000F0D3
:105A7000AFBFFFF7D5F900F0ABBFB2783E4B022ABB
:105A800000F0E580032A00F0E780002A40F0218141
:105A90005B78512B00F0BB8037D8472B00F0A580F6
:105AA00019D8432B00F09A800DD8412B00F090803C
:105AB00000F29080402B40F00A8140F2FF7001F02C
:105AC00013FC786007E1452B2C4A00F08A8000F235
:105AD0008A80D36980E04C2B00F090800AD8492B53
:105AE00000F08980C0F083804B2B40F0F080234B86
:105AF000DB7871E04F2B00F0848000F285804D2B25
:105B000040F0E5801D4B5B7D66E0802B00F08F80D0
:105B100036D8552B00F0818005D8532B174A78D002
:105B200079D8136A58E0592B7AD05A2B7BD0572B4F
:105B300040F0CD80114B93F827304DE03F2D0020F1
:105B40003C2D0020532D0020442D0020402D00200E
:105B50003D2D00203E2D00204C2D0020342D002016
:105B6000382D0020422D0020482D0020502D0020EF
:105B7000412D0020342D002088280020080000201E
:105B8000842B5BD00BD8822B984A53D054D8137DEA
:105B9000B3F1040CDCF1000353EB0C031CE0F02B1D
:105BA0004ED00DD8852B40F09280904A9049536892
:105BB0004B4303F540533933536023F000430BE06C
:105BC000FE2B3DD0FF2B40F082808A4B1B783AE0C1
:105BD000894B36E0884B5B7863607CE0864B1B79B1
:105BE000FAE75379F8E7D368F6E7834B5EE0824B38
:105BF00093F82630F0E7804BDB7D24E07E4B9B78EA
:105C0000EAE77D4B5B7EE7E77B4B9B7DE4E77A4BE6
:105C10000EE01369E0E7937EDEE7774BDB7EDBE7A0
:105C2000754B9B8CD8E7744B93F82830D4E76F4BB7
:105C30001B7DD1E79369CFE71368CDE76F4B32E067
:105C40006F4B1B78C8E7003318BF0123C4E75A78AD
:105C50006C4B53F82230BFE75B78282B28D00FD845
:105C6000022B22D005D8EBB1012B30D1664B5B68FB
:105C7000B2E7092B2FD0272B29D1634BDB68ABE789
:105C80002B2B1BD006D8292B15D02A2B1FD15E4BCE
:105C90009B69A1E72D2B17D013D32E2B17D15A4B6D
:105CA0009B6A99E7584B1B6896E7574B9B6893E7AD
:105CB000554B1B6990E7544B5B698DE7524BDB6991
:105CC0008AE7514B1B6A87E74F4B5B6A84E70323E4
:105CD00000E0042323704D4B1B78002B00F07886E6
:105CE0004B4B62681A604B4B2AB91A6842F00802A3
:105CF0001A6000F06DBE1A6822F008021A6000F007
:105D000067BEB378022B15D17378372B0ED83D4977
:105D100003F5A770800001EB8301042201F0AEFAC5
:105D200000F056BE7378142B40F2D8820323237000
:105D300000F04EBE04233B7000F04ABEB378022B45
:105D40000ED1354B5B78372BF0D82E4903F5A77071
:105D5000800001EB8301042201F0CCFA00F038BE90
:105D600004233B7000F034BEB378002B7FF4EEAA1E
:105D70007378012B10D002D3022B12D029E002F04D
:105D80001DFF28B9244B987804F0A2F800F020BE3B
:105D900006233B7000F01CBE002004F0A1F800F0C8
:105DA00017BE002004F0A4F8184B78601B78002B75
:105DB00000F00E86164B1860164B1A6820B942F098
:105DC00008021A6000F004BE22F008021A6000F017
:105DD000FFBD03233B7000F0FBBDB37813B1022B72
:105DE0001CD036E0FEF72EFB00F0F2BDD004002000
:105DF0006D4EC641F628002008000020F82800203B
:105E00008C2D0020082900205C2D0020F728002080
:105E1000E82800209028002088280020974B5B78F5
:105E2000072B0AD820B91846FEF776FA00F0D0BD45
:105E30001846FEF77DFA00F0CBBDFF2B7FF476AF5E
:105E4000471C0ABF8E4BC0B21878FEF77DFA00F0EF
:105E5000BFBD04233B7000F0BBBDB378012B23D042
:105E600005D3022B24D17078FEF7A2FA0DE07078EA
:105E7000082802D8FEF779FA07E00A2801D10023A2
:105E80000BE00B2803D1FEF793FC606012E00C28B6
:105E900005D17C4B9B68C3F3800363600AE0FF2855
:105EA00008D1FEF797FAF0E7707802F097F8ECE780
:105EB00004233B70744B1B78002B00F08985704BDA
:105EC00062681A60714B2AB91A6842F008021A60B7
:105ED00000F07EBD1A6822F008021A6000F078BD5A
:105EE0007278674B092A27D8DFE802F005080B0E05
:105EF00012181B1E21251A6810441CE01A68101A7B
:105F000019E01A68504316E01A6892FBF0F012E0AC
:105F10001A6892FBF0F100FB11200CE01A681040A7
:105F200009E01A68104306E01A68504003E01A6856
:105F3000D2431A6000E018601A68544B2AB91A68F4
:105F400042F008021A6000F043BD1A6822F008020D
:105F50001A6000F03DBD4A4B1A684C4B82421968EA
:105F600004DD21F0030141F0040108E00BBF21F042
:105F7000060121F0050141F0010141F00201196023
:105F80002AB91A6842F008021A6000F021BD1A68A6
:105F900022F008021A6000F01BBD73780C2B00F28F
:105FA0001785DFE803F0071019222B343E475059BC
:105FB00062778000354B1B681E0740F10985344B22
:105FC000986100F005BD314B1B681D0700F100858D
:105FD0002F4B986100F0FCBC2C4B1B68DC0740F198
:105FE000F7842B4B986100F0F3BC284B1B68D90752
:105FF00000F1EE84264B986100F0EABC234B1B684D
:106000005A0740F1E584224B986100F0E1BC1F4B38
:106010001B6813F0050F00F0DB841D4B986100F046
:10602000D7BC1A4B1B689B0740F1D284184B986170
:1060300000F0CEBC154B1B689F0700F0C984144BC1
:10604000986100F0C5BC114B1B68DE0640F1C084AE
:106050000F4B986100F0BCBC0C4B1B689D0640F1D7
:10606000B7840B4B986100F0B3BC084B1B685C060F
:1060700040F1AE84064B986100F0AABC882800204D
:10608000E8280020000C0140F7280020902800207C
:10609000D00400209C4B1B68190640F199849B4B4F
:1060A000986100F095BC984B1B68DA0540F190842C
:1060B000964B986100F08CBCDA69072A00F288845C
:1060C000511CD961996903EB82021162986100F059
:1060D0007FBCDB698D4A002B00F07A84013BD361E1
:1060E00002EB83031B6A936100F072BC73782E2B62
:1060F00004D8874A0121D15400F06ABCFF2B7FF4F9
:1061000015AE824B012283F8402000F061BC737809
:106110002E2B04D87E4A0021D15400F059BCFF2B0D
:106120007FF404AE794B002283F8402000F050BC8D
:10613000764C94F8413083B9431C4FF00A0304D1E4
:10614000744A10684343636401E05843606401F09B
:10615000BDFE0123A06484F841306B78042B00F26B
:106160003784DFE803F003416896190001F0AEFEC2
:10617000A26C616C801A80EAE072A2EBE0728A4243
:10618000624B04D9002283F8412000F021BC9A69B7
:10619000013A9A6100F01CBCA87803F0A9FE40B94E
:1061A000594B84F841001A6822F010021A6000F07E
:1061B0000FBC636C554D9BB101F088FEAB6C6A6CF3
:1061C000C01A80EAE073A3EBE073934208D900237E
:1061D00085F841304C4B1A6842F010021A60F7E320
:1061E000A369013BA361F3E303F096FB064640B1CC
:1061F000002384F84130444B1A6822F010021A60E0
:10620000E6E3636C414D93B101F060FEAB6C6A6CE8
:10621000C01A80EAE073A3EBE073934207D93A4BCC
:1062200085F841601A6842F010021A60D0E3A36951
:10623000013BA361CCE3384B5A7E384B9B6812B9C3
:106240005F070BD501E05E0708D4002384F84130D6
:106250002D4B1A6822F010021A60B9E3636C2B4DC3
:106260009BB101F033FEAB6C6A6CC01A80EAE0733C
:10627000A3EBE073934208D9002385F84130224B09
:106280001A6842F010021A60A2E3A369013BA361FD
:106290009EE3214B5A7E214B9B6812B99D0702D584
:1062A000D3E79807D1D5636C184D9BB101F00EFE72
:1062B000AB6C6A6CC01A80EAE073A3EBE0739342A4
:1062C00008D9002385F841300F4B1A6842F01002BC
:1062D0001A607DE3A369013BA36179E3B2780ABB4D
:1062E0000D4A0F49927E41F82300002A00F0708386
:1062F000002B00F06D8303F28510800001EB830119
:10630000042200F0BBFF63E390280020D0040020AB
:106310009E2D0020E82800200800002000080140F1
:1063200094280020FF2A7FF411A863B94FF4C364B6
:106330009249204621440422043400F09FFFB4F522
:10634000CD6FF5D144E38E4903F28510800001EB57
:106350008301042200F092FF3AE37378142B3FF696
:10636000E5AC884A9278B2B9854A52F82320864B28
:106370007A601B78002B00F02B83844B1A60844BCF
:1063800022B91A6842F008021A6021E31A6822F062
:1063900008021A601CE3FF2A7EF4D8AF63B94FF4F9
:1063A000C3647649204621440422043400F0A2FF4D
:1063B000B4F5CD6FF5D10BE3714903F28510800080
:1063C00001EB8301042200F095FF01E37678142E9F
:1063D0003FF6ACACAB786B4F190619D5DA0704D58C
:1063E00003F064FA664B43F826006A4B9B7E002B51
:1063F00000F0EE826B78002B00F0EA82604903F235
:106400008510800001EB8301042200F037FFDFE2FA
:10641000002B7EF49BAF03F049FA5E4B584A9B7EFB
:1064200042F82600002B00F0D3827B78002B00F08E
:10643000CF82B97803F285100844194402EB810138
:106440008000042200F01AFFC2E272784F4B0A2A41
:1064500042D8DFE802F0060B11161C24292E33382F
:106460003C004D491A6809680A4403E04A491A6821
:106470000968521A1A602FE047491A6809684A43A6
:10648000F8E745491A68096892FBF1F2F2E7424AD7
:106490001968126891FBF2F002FB1012EAE73E4A1B
:1064A00011681A680A40E5E73B4A11681A680A430E
:1064B000E0E7394A11681A684A40DBE7364A116852
:1064C000C943116008E01A6833490A6004E0324A9F
:1064D00018681168106019601A682D4B22B91A6883
:1064E00042F008021A6073E21A6822F008021A6089
:1064F0006EE2264B1B68C6F80330FEF729FA67E206
:10650000224B1B68C6F80330FEF78AFC60E2737802
:10651000052B00F25D82DFE803F003090F151B2154
:106520001B4B1A6802F00F021A6051E2184B1A68EE
:1065300022F010021A604BE2154B1A6822F020027A
:106540001A6045E2124B1A6822F040021A603FE2DC
:106550000F4B1A6822F080021A6039E20C4B1A685D
:1065600022F480721A6033E273782E2B3FF6DEAB92
:106570000A4A02EB8303D8642AE200BF802200208B
:106580009428002088280020F7280020E8280020F0
:10659000902800200800002004290020D0040020BA
:1065A000AA4BAB49D3F808210A60D3F80C21A949BA
:1065B0000A60D3F81021A8499A61D3F814210A601F
:1065C000D3F81821A54983F84120D3F81C219A64F7
:1065D000D3F820215A6493F82421885C08B1012063
:1065E0008854002283F82821F2E1B378002B7EF44E
:1065F000ADAE7378142B3FF699AB954A1168984A63
:1066000042F82310E4E101F07DFDE1E101F07CFDC1
:10661000DEE101F08BFDDBE101F089FDD8E101F065
:1066200087FDD5E101F085FDD2E1737813B1012B2F
:1066300004D00BE0854B01221A75C9E1B0F55B7FF0
:10664000BEF484AE814A13759061C1E103233B70AF
:10665000BEE17E4B02221A75BAE17C4A4FF0FF3050
:1066600002F14C0343F821007C48002343540131DC
:106670002F29F2D113759361D36182F84130744AA6
:106680001360744A1360744A1360A1E1754B1B7D5B
:106690009B0709D4B0F55B7FBEF458AE6B4B042268
:1066A0001A75C3F82C0193E108233B7090E16E4BFF
:1066B00001221A706B4B6D4C9A78B0F55B7F22709B
:1066C00025D21B7D13F0010521D1694600F027FE7C
:1066D0009DF80030257263709DF80130A3709DF81D
:1066E0000230E3709DF8063023719DF80530637128
:1066F0009DF80430A3719DF80330E3710123E15C40
:10670000227A01330A44082B2272F8D160E1012376
:106710000021E1540133082B544AF9D11378137244
:1067200056E17378012B1DD00AD3022B2BD14E4B8F
:1067300001221A704B4B4D4A9B781370002319E0CD
:10674000494B01221A70474B484A9B781370484BBB
:10675000186800230133C11811F8011C082BD1540B
:10676000F8D135E10322FA717B71FD222A23BA7137
:106770003B712DE13F490133194411F8091C082BE5
:10678000D154F7D124E103233B7021E17378032B2B
:1067900000F21E81DFE803F0020E191D2B4B1A7D5B
:1067A000FA7193F84120D3F82C31BA711A0A7A7130
:1067B0003B710DE1254B1A7DFA7193F841209B69DD
:1067C000BA711A0A7A713B7102E1214B1B687B6036
:1067D000FEE0204B1B687B60FAE07378002B40F0F2
:1067E000F780254B9978002940F0F28040F2D2439F
:1067F000984240F0ED8040F2FF7000F026FD00F07E
:1068000095FD0120FDF705FEE2E072781B4B02B119
:1068100001221A70EA781A4B1A700C4B93F8301157
:10682000184B1970184900230B7018490B70184B3E
:1068300019780A431A70CBE0044B012283F8312106
:10684000C6E0757835B3012D33D03FE0D004002089
:10685000E828002004290020902800209E2D0020F8
:106860009428002008000020EC280020ED280020BB
:10687000000000200040000888280020102D002083
:10688000242D0020962D00201E2D0020CD2D00202F
:10689000112D0020042240F2FB70694600F02AFD11
:1068A000009BD6F803209A4206BF01237B607D60DF
:1068B0008EE0B3782A2B06D140F2FB7045490422C2
:1068C00000F0DCFC84E003233B7081E003233B7099
:1068D0007EE07378032B3CD8DFE803F008022D3804
:1068E0003D4A0023D2F83411154610E03A4BD3F854
:1068F0003421092A07D8511CC3F8341103EB820351
:10690000C3F8380164E009233B7061E001338B4236
:106910005ED0324A9E0052F823408442F6D132447F
:10692000481E834204D25068013342F8040BF7E753
:10693000C5F834014CE0284A0023C2F83431274A14
:10694000002199500433282BF9D141E00A237B60C0
:106950003EE003233B703BE07378812B38D1B27863
:106960001F4B922A34D19A79A32A31D15A79B42A69
:106970002ED11A79C52A2BD1DB78D62B28D1194BE9
:1069800008221A61FDF74CFD05F01CFA002005F005
:10699000EDFE0021144804F00AFC134804F06CFBDF
:1069A000124803F0DFFE04F047FC4FF0804005F092
:1069B00033FF0020FDF72DFD0AE040F2D24398425C
:1069C00006D1054B012283F8602101E002232370E8
:1069D00003B0F0BD8B280020D00400200806002062
:1069E00088280020000801400800024000240140DF
:1069F0002D49002370B50B602C492D4A0B602D49A1
:106A00009361D3610B6082F8413082F8403082F8A4
:106A100028311546284A4FF0FF3142F82310274A03
:106A20000024D45401332F2BF4D1254E307B02F0B7
:106A3000B7FFF07A02F0DCFF2346224A002199508A
:106A40000433B3F5806FF8D11F4EB37E13B9F37ED4
:106A50006BB118E04FF4C3641C4920462144042262
:106A6000043400F047FCB4F5CD6FF5D1EFE74FF4F7
:106A7000A7641749204621440422043400F03AFC5C
:106A8000B4F5C36FF5D1337903F0EF02012A01D0D9
:106A9000212B01D1012300E0002385F86131737DB2
:106AA00003B101232B7570BDE828002004290020C4
:106AB000D0040020902800201C0500209E2D0020DE
:106AC000342D00200829002008000020802200200A
:106AD000D0230020F7B50F4E0F4CC6F803300F4BF4
:106AE00086460F46B270002294E803001A708DE8C3
:106AF000030086F800E07770FEF73EFB21786368BC
:106B0000074A82F862119DE8030084E803001846F2
:106B100003B0F0BD88280020FC280020F7280020C2
:106B2000D0040020014B93F862017047D00400208C
:106B3000F7B51F4E024653780C4696E803008DE8E1
:106B400003001C4900270B7093786D464B70D37877
:106B50008B7013798B7153794B7193790B71D37956
:106B6000CB70154B1F70FEF707FB144B197833469B
:106B700071B9217032786170A2707278E270F27926
:106B80002271B27962717279A2713279E27109E08F
:106B9000012907D13A460A4911444978A1540132E2
:106BA000082AF8D195E8030083E8030003B0F0BD9C
:106BB000FC28002088280020F7280020EC2800204E
:106BC000ED2800202DE9F047714B88B01B78714CFF
:106BD00013B994F8633163B16F4B1B78062B08D05F
:106BE0000A2B06D003F0EF030F2B1CBF002384F801
:106BF000303194F83031694E5A1E012A40D8684924
:106C0000012BCA6814BF082307238DF8003094F8BD
:106C10006431019232788DF8013000238DF8023012
:106C2000C2B98B688DF80F208DF808305D4B19784C
:106C30008DF8091059788DF80A10D9798DF80B1054
:106C400099798DF80C1059791B798DF80D108DF804
:106C50000E300AE0012A08D15349013308AA595CD1
:106C60001A44082B02F8191CF6D1504B1B78002B44
:106C700058D1684601F062F8002800F0C58251E062
:106C8000032B25D1434B93F86151EDB933788BB980
:106C9000434F444DB87897F801802A788044904457
:106CA0006A789044EA799044AA7990446A79904449
:106CB0002A791AE0012B35D13B4B585D013500F0A4
:106CC0001FFD092DF8D12DE0364803F0D1FC29E055
:106CD000042B27D1324F334DB87897F80180002329
:106CE00001226B702A706B608044904400F008FDB4
:106CF000787800F005FD287800F002FD687800F053
:106D0000FFFCE87900F0FCFCA87900F0F9FC687958
:106D100000F0F6FC5FFA88F8287900F0F1FC4046B4
:106D200000F0EEFC224BDFF884801A789946002AA6
:106D30006BD0204B204D1B78002B62D0022B3DD90D
:106D4000032B5ED1164F2A78B87897F801A08244B9
:106D50000AF10A0A924400F0D3FC787800F0D0FCE3
:106D6000802000F0CDFC8A2000F0CAFC002000F05A
:106D7000C7FC002000F0C4FC002000F0C1FC5FFA5A
:106D80008AFA287800F0BCFC504600F0B9FC38E0E4
:106D9000F6280020D004002088280020EC280020BD
:106DA00008000020FC280020ED280020082D0020ED
:106DB000CD2D0020962D00201E2D0020994A2978E7
:106DC00093688DF81E108DF8183080238DF81930D7
:106DD0008A238DF81A3000238DF81B308DF81C3073
:106DE0008DF81D308DF811308DF81230D3680721E1
:106DF000059398F800308DF8101013B904A800F02E
:106E00009DFF00232B7089F80030002384F8303177
:106E1000337084F8633194F8603113B10120FDF7C9
:106E2000F8FA94F83121804B52B193F86121D2F1F4
:106E3000010238BF002283F86121002283F831214A
:106E400098F80030002B44D1684600F0C1FF0028BC
:106E50003FD09DF80030062B3BD9744B9DF808209D
:106E60001A709DF809205A709DF80A209A709DF8B2
:106E70000B209A719DF80C205A719DF80D201A7103
:106E80009DF80E20DA709DF8013084F86431654B6E
:106E90001A69019B934203D1634B012283F863215A
:106EA00001F014F8624B00221860624B1A709DF8D2
:106EB0000030227D072B0CBF0123022384F83031E0
:106EC000531E012B5C4B02D9052A40F09180002211
:106ED000A5E094F86151002D70D104A800F02AFCBF
:106EE00000286BD000F044FC10B14F4B83F8655183
:106EF00094F865119DF810004A1CD2B22144092A69
:106F0000494B84F8652181F8660140F09D8000229C
:106F100083F86521434A93F866315178994207D046
:106F200092F82710002900F08F808B4240F08C806F
:106F300092F827209A4204BF012384F8633100238A
:106F40001A46394D05F5B371595C01330A44082BD3
:106F5000D2B2F6D195F86E3193422BD1334B95F8DE
:106F600067211A7095F868215A7095F869219A700E
:106F700095F86A219A7195F86B215A7195F86C21F0
:106F80001A7195F86D21DA7000F0A0FF2B4B2C4A96
:106F90001860297D00231370032285F830214A1ED2
:106FA000012A85F86531244A02D9052918BF012331
:106FB000137049E0042385F8303145E094F86131DD
:106FC000194DCBB1194803F01BFAA8B100F07EFFB0
:106FD0001A4B1B4A186000231370032285F83021D6
:106FE0002A7D511E01291946134B03D9052A01D0C8
:106FF000012214E0197027E0237D0B4D013B012B8A
:1070000022D8A869B0F55B7F1CD2431C0749AB614D
:1070100000F085F9092385F83031074B01221A70F9
:1070200012E000BF08000020D004002088280020C3
:10703000882D0020092D0020F7280020902D002009
:10704000952D002000232B75237D714D042B04D139
:10705000704E3278170640F1AD8094F8303113F05D
:10706000FB0F05D0082B03D0062B01D0FEF784F8C8
:1070700094F83031092B79D100F028FF644A664D2D
:1070800092682B68801A80EAE072A2EBE0729A4262
:1070900008D9624B1A78012A04BF02221A7000F044
:1070A00015FFA06000F012FFE3686A68C01A80EA6A
:1070B000E073A3EBE073934208D9584B5A78012A46
:1070C00004BF02225A7000F001FFE06000F0FEFEF3
:1070D0002369AA68C01A80EAE073A3EBE0739342C5
:1070E00008D94E4B9A78012A04BF02229A7000F008
:1070F000EDFE206194F84030002B37D0444B93F8DC
:107100002821002A32D145498B5C022B2BD1404BE0
:1071100003F14C0050F82200451C22D0404983F86E
:10712000242109680022C3F808113E490968C3F800
:107130000C1199699861C3F810113B490968C3F8AB
:10714000141193F8411083F84120C3F81811996C79
:107150000122C3F81C11596C83F82821C3F82011AF
:1071600004E000238B5401322F2ACCD194F8301143
:10717000274B092904D11A7D022A04BF05221A755A
:10718000D4F83421224B002A3ED009293CD1197D64
:10719000012939D1986900231D4901F59C7454F8DF
:1071A0002340A04202D105230B752DE00133934209
:1071B000F2D129E095F8303113F0FB0F24D0082BE1
:1071C00022D0062B20D0D5F82C01184CD6F803304D
:1071D000B0F55B7F6270636012D2314600F098F8C0
:1071E000D5F82C01314600F0C9F830B1D5F82C3172
:1071F0000133C5F82C31652300E00723237003E039
:107200000723237000232B7508B0BDE8F08700BF6B
:10721000D0040020882800205C2D00209E2D002016
:10722000E82800200429002090280020FC280020C5
:1072300010B500F04BFE044600F048FE001B00288D
:10724000B8BF40420628F7DD10BD07B5094B8DF8E1
:1072500005001954030A8DF804308DF80610032236
:1072600001A9A023044802F00DFFFFF7E1FF03B0DE
:107270005DF804FB4006002000540040F0B50023F8
:107280008BB00E461546AB4205D0154AF15C024460
:10729000D1540133F7E700231C46AC421DD0315DC9
:1072A0000AAA1A4402F8221C5A1C1718F90602D01E
:1072B000691E8C420ED1020A8DF804208DF805005B
:1072C000DA1C01A9A023074802F0DCFEFFF7B0FF9B
:1072D0003846002201341346DFE70BB0F0BD00BF93
:1072E0004006002000540040014B185C704700BF6E
:1072F0004006002010B50023934205D0034C0444FF
:10730000E45CCC540133F7E710BD00BF4006002019
:10731000C0EBC00000F500600722FFF7AFBFC0EB75
:10732000C00000F500600722FFF7E4BF30B54FF45E
:1073300000628BB00F49002353540132B2F5005F55
:10734000F8D101AD00245C550133222BF9D1230A79
:107350008DF804308DF8054029462222A0230648E6
:10736000203402F08FFEFFF763FFB4F5005FEED12B
:107370000BB030BD40060020005400401FB5C0EBEC
:10738000C00000F50060030A0C468DF804308DF84B
:10739000050001A90222A023114802F073FE072272
:1073A000A0230F4802A902F0D9FD9DF808202378F8
:1073B0009A4211D19DF8092063789A420CD19DF828
:1073C0000A20A3789A4207D1DDF80B00D4F80330E5
:1073D000C31A5842584100E0002004B010BD00BF5D
:1073E0000054004013B50A4C00238DF804308DF88A
:1073F000053001A920460222A02302F043FE2046C8
:1074000004494FF40052A02302F0A8FD02B010BDC1
:10741000005400404006002013B5FFF7E3FF254B62
:1074200093F8FF37422B02D1234B1B78ABB340F2CA
:10743000FF700021FFF709FFFFF778FF00201F49C9
:107440004022FFF71BFF4FF480701D49B422FFF765
:1074500015FF40201B492022FFF710FF0023019356
:107460004FF4C364204601A904220434FFF706FF49
:10747000B4F5FF6FF6D1002301934FF4A7642046C3
:1074800001A904220434FFF7F9FEB4F5C36FF6D165
:1074900040F2FF704221FFF7D8FE0020074940224A
:1074A000FFF728FF402008492022FFF723FF02B002
:1074B00010BD00BF400600202C2D00200800002039
:1074C000FCEE0008DCEE0008342D002030B5054647
:1074D00087B0544805F08CFE4FF48040012104F041
:1074E00019FF0420002104F049FA03238DF8063027
:1074F00018230DEB03048DF807304FF4007324F8C4
:10750000143D4948214604F0AAF948238DF8073074
:1075100045484FF480632146ADF8043004F09FF9EC
:1075200002A805F0F3FE0B2D25D8DFE805F02406B0
:10753000090C0F1215181B1E20224FF461531CE07A
:107540004FF4964319E04FF4E14316E04FF416432D
:1075500013E04FF4614310E04FF496330DE04FF425
:10756000E1330AE04FF4613307E0304B05E0304B84
:1075700003E0304B01E04FF416530293FCF763FF36
:10758000B0F5827F02D3029B5B08029302A92548D3
:1075900005F078FE2523002401258DF8003068468B
:1075A00007238DF801308DF802408DF8035004F068
:1075B00045FC1C4840F2FF3105F090FF2246194877
:1075C000282105F0D0FE2A46164840F2277105F022
:1075D000CAFE2A46134840F2266105F0C4FE2A4638
:1075E000104840F2255105F0BEFE22460D4840F2FB
:1075F000244105F0B8FE22460A4840F6460105F04F
:10760000B2FE2246074840F66A1105F0ACFE22465B
:107610000448602105F0A7FE0248294605F097FEC0
:1076200007B030BD003801400008014090D0030091
:1076300020A1070040420F00684620F007018D4658
:107640002A4919B50B889C061AD5294BDB68D80541
:1076500001D58B8814E0274B1A6858680132202A1C
:1076600008BF0022824205D01C6888881919C0B260
:1076700008721A60204A0A2111609A6A1F4B1A6028
:107680001A4803881A061CD51C4B1A68CAB9194B2C
:10769000DC6A196B8C4210D015494FF480740C6170
:1076A000196B4C1C1C63194491F83410C9B28180C9
:1076B000196B202905D11A6303E040F2277105F008
:1076C00052FE0A4803885B060CD540F2266105F09D
:1076D00029FF084B1A6BDB6A9A4203D1044B4FF423
:1076E00080725A61BDE819408546704700380140F4
:1076F0000008014040260020D42D0020D02D00207D
:107700000A4BDA6A196B0132202A08BF00228A422A
:107710000AD0D96A194481F83400DA62044840F288
:107720002771012205F01FBE704700BF40260020D0
:10773000003801400A4B59681A6891420BD05A68C8
:10774000511C59601A44127A02705A68202A04D1D6
:1077500000225A6001E0002070470120704700BFFE
:1077600040260020014B9862704700BF4026002051
:10777000044B1A7802F0FF0012B100221A700120A7
:10778000704700BFD82D002008B5FCF749FE044B18
:1077900000225A601A60BDE80840FCF73FBE00BFF7
:1077A0004026002010B5441E14F8010F10B1FFF759
:1077B000A7FFF9E710BD00BF684620F007018D461E
:1077C00031B5264C264B25681B680135082D08BFAE
:1077D00000259D4286B04FF0000037D001A903F08C
:1077E0002DFB9DF80C302268042B1E4B03EB02127C
:1077F00006D1012151702168029A03EB011105E0C5
:10780000002151702168019A03EB01114A609DF833
:107810000D20022A226808BF012103EB021218BFC3
:107820000021917022689DF80E10120199540022D7
:10783000216801A8104403EB01111144C07A013200
:10784000082A0872F4D1054B1D6001E003F0DCFA50
:1078500006B0BDE831408546704700BF682E002065
:10786000DC2D0020E82D0020684620F007018D4621
:1078700031B5264C264B25681B680135082D08BFFD
:1078800000259D4286B04FF0010037D001A903F0DA
:10789000D5FA9DF80C302268042B1E4B03EB021224
:1078A00006D1012151702168029A03EB011105E014
:1078B000002151702168019A03EB01114A609DF883
:1078C0000D20022A226808BF012103EB021218BF13
:1078D0000021917022689DF80E1012019954002227
:1078E000216801A8104403EB01111144C07A013250
:1078F000082A0872F4D1054B1D6001E003F084FAF8
:1079000006B0BDE831408546704700BF682E0020B4
:10791000DC2D0020E82D0020684620F007018D4670
:1079200031B52A4B2A4A1968126886B0914204D1AF
:107930000120002103F0A2F943E01A68254901EB78
:107940000212507800F0FF0248B104228DF80C209A
:10795000002201921A6801EB0212526806E01868D0
:107960008DF80C2001EB00104068019002921A681B
:1079700001EB0212927802F0FF001AB102228DF898
:107980000D2001E08DF80D001A6812018A5C8DF857
:107990000E2000221C680D4801EB04141444257AC3
:1079A00001AC14440132082AE572F3D103680133B3
:1079B00003600368082B04BF0023036001A803F0E1
:1079C00069F906B0BDE8314085467047E42D0020D6
:1079D000E02D00206C2E0020F0B501388BB00F4652
:1079E0001546072845D8DFE800F03C342C241C4419
:1079F0001404FCF728FDB0F5827F14BF0223042392
:107A0000ADF8163005238DF8143000238DF81530AD
:107A10003FE0FCF718FDB0F5827F14BF022304237A
:107A20002EE0FCF710FDB0F5827F14BF0823102371
:107A300026E0FCF708FDB0F5827F14BF0A2314236B
:107A40001EE0FCF700FDB0F5827F14BF142328234D
:107A500016E0FCF7F8FCB0F5827F14BF32236423F4
:107A60000EE0FCF7F0FCB0F5827F14BF6423C8235E
:107A700006E0FCF7E8FCB0F5827F14BF042308237E
:107A8000ADF816300C238DF8143001238DF8153025
:107A900000238DF8133003F003F84FF0007001213C
:107AA00004F044FC0120014604F034FC08200121CC
:107AB00004F030FC0820002104F044FC4FF4EA10EC
:107AC000012103F05BFF03238DF8063018230AAC75
:107AD0008DF807304FF4007324F8243D2146784890
:107AE00003F0BDFE042321468DF8073074484FF49F
:107AF000807300240126ADF8043003F0B0FE03A823
:107B00008DF812408DF80C408DF80D608DF80E4008
:107B10008DF80F408DF810608DF8116002F0CDFFE8
:107B2000B7F5006F8DF818408DF819408DF81A6080
:107B30000FDA7B01ADF81C304FF6FF73ADF81E4035
:107B4000ADF82030ADF82230ADF824408DF8266035
:107B50000DE04FF6FF73ADF81C40ADF81E40ADF8D8
:107B60002030ADF82230ADF824408DF8264006A82C
:107B700003F002F8012300228DF818308DF8192047
:107B80008DF81A3095B1B5F5006F0FDA6901ADF8CF
:107B90001E204FF6FF72ADF81C10ADF82020ADF896
:107BA0002220ADF824308DF826300DE04FF6FF711D
:107BB000ADF81C20ADF81E20ADF82010ADF8221055
:107BC000ADF824308DF8262006A802F0D5FF022358
:107BD0008DF818307B13FF0047F0040700260124BE
:107BE000ADF81E7006A84FF6FF77ADF81C308DF883
:107BF00019608DF81A40ADF82070ADF82270ADF81C
:107C000024608DF8264002F0B7FF0323B5428DF8BB
:107C100018308DF819608DF81A4010DD6B13ED00E7
:107C200045F00405ADF81C30ADF81E50ADF82070DD
:107C3000ADF82270ADF824408DF826400CE0042306
:107C4000ADF81C60ADF81E30ADF82070ADF82270B4
:107C5000ADF824408DF8266006A802F08DFF0124BF
:107C600007260025142302A88DF808308DF8096036
:107C70008DF80A508DF80B4004F0E0F8152302A8A7
:107C80008DF808308DF809608DF80A508DF80B409A
:107C900004F0D4F8132302A88DF808308DF8096099
:107CA0008DF80A508DF80B4004F0C8F821460220E8
:107CB00002F0E4FF1020214602F0E0FF0BB0F0BD1F
:107CC000000C014037B50220002102F0D7FF102040
:107CD000002102F0D3FF0021012002F0CFFF002499
:107CE0000725142301A88DF804308DF805508DF870
:107CF00006408DF8074004F0A1F8152301A88DF87F
:107D000004308DF805508DF806408DF8074004F0DA
:107D100095F8132301A88DF804308DF805508DF8DF
:107D200006408DF8074004F089F802F0B9FE4FF0E4
:107D30000070214604F0FAFA03B030BDF0B5437884
:107D400087B00446426833B104238DF80C30002319
:107D50000292019303E08DF80C3001920293A37814
:107D600003B102238DF80D3023788DF80E300023F7
:107D7000E11801AA1A44097A0133082BD172F7D10C
:107D800001A802F087FF042816D10E4F0E4B3D6864
:107D90001B680135082D08BF00259D420ED03E68A6
:107DA0000A4B03EB061694E80F0086E80F0001204B
:107DB00001463D6002F062FF012000E0002007B0B4
:107DC000F0BD00BFE02D0020E42D00206C2E00202F
:107DD00030B50D4B0D4C054622681B689A420ED0FB
:107DE00023685A1C22600A4A02EB03130FCB85E872
:107DF0000F002368082B04D10023236001E000203A
:107E000030BD012030BD00BF682E0020DC2D0020D9
:107E1000E82D0020684620F007018D4601B5BDE839
:107E200001408546704700BF684620F007018D4637
:107E300001B5124B19781A4679B15B68013353606A
:107E40000F4B1968013119600E4B196811B119688F
:107E5000013919600023137001E001221A700A4BE6
:107E60001A683AB11A68013A1A601B6813B9074BCD
:107E700001221A70BDE80140854670479426002013
:107E8000F8280020D02D0020D42D0020D82D00204F
:107E900008B5042004F044FCFCF7D5FAB0F5827F65
:107EA000ACBF4FF47A504FF4FA5004F045FC012077
:107EB00004F048FC04480321002204F095F8BDE8D2
:107EC0000840012004F052BC9AC30200014B5868DC
:107ED000704700BF94260020F0B593B0002403261D
:107EE000394801A9ADF804608DF806608DF80740A7
:107EF00003F0B5FC0120014604F000FA01214FF423
:107F0000007004F007FA314803F0B6F8304B02274E
:107F10000793304B2D48089380230C934FF48073C4
:107F20000D934FF480630E9320230F9307A94FF412
:107F30000053109309940A970B94119403F00CF9D1
:107F40002248012103F033F901254FF46023224830
:107F500002A9049302948DF80C508DF80D500594ED
:107F60008DF8187002F02AFC1B4809212A46334676
:107F700002F09CFC3346184808213A4602F096FC71
:107F8000224615484FF4FC6102F057FC124829467E
:107F900002F04AFC1048294602F03DFC0E4802F06F
:107FA00055FC0D4802F057FC0028FAD10A4802F0AF
:107FB00056FC094802F058FC0028FAD10648012175
:107FC00002F056FC13B0F0BD000C01400800024066
:107FD0004C2401409C26002000240140F8B50028D4
:107FE0004ED0092850D1364B588880B206F022F87E
:107FF00005F02CFC0022334B05F07CFC24A3D3E9D4
:10800000002305F077FC04460D4622462B4620A1AE
:10801000D1E9000105F0BAFA1FA3D3E9002306460F
:108020000F462046294605F08FFD02460B46304696
:10803000394605F089FD05F0F7FE05F007FC002242
:10804000214B05F081FD06F0A7FC15A3D3E9002321
:1080500005F050FC14A3D3E9002305F099FA024679
:108060000B4613A1D1E9000105F06EFD12A3D3E97F
:10807000002305F08BFA05F0D7FE06F033F8F8BDC3
:108080000F4B188880B2F8BD0020F8BDAFF3008018
:108090006666666666660A409A999999999901405A
:1080A000C3F5285C8FA272400000000000FEAA40C9
:1080B0009A999999FD6F2F41C3F5285C8F127140F1
:1080C0009C2600200000303F00002440AFF30080D9
:1080D000704710B5FFF7FAFE074C2368C01AB0F5D9
:1080E000FA7F07D9054BDA6882F40042DA60FFF7BD
:1080F000EDFE206010BD00BFEC2E002000100140FE
:108100007047704770477047054B064AD3F8031015
:10811000054B09B9928800E0128992B25A60704703
:1081200088280020006C0040FC2800207047704721
:1081300070477047F8B5054601F054FC20B1284659
:10814000BDE8F84001F068BCFCF76AF9274B102243
:108150005A611E462648022104F09EFA0028F9D0F2
:108160002348290C04F044FA2148012104F094FA30
:108170000028F9D01E4804F03DFA1E4C0002206091
:108180001B48022104F088FA0028F9D01848C5F3EA
:108190000F2104F02DFA1648012104F07DFA002881
:1081A000F9D01348276804F025FA384307022760FE
:1081B0000F48022104F070FA0028F9D00C48E9B207
:1081C00004F016FA0A48012104F066FA0028F9D0F2
:1081D0000748256804F00EFA284310230509336187
:1081E0002560BDE8F840FCF719B900BF0008014060
:1081F00000300140A026002038B5484C0B2303FB7B
:10820000004203FB004311790433032984BF032197
:1082100011719A78032A84BF03229A700B2303FBFF
:10822000004203FB0043117A04320F2984BF0F215F
:1082300011715A7A0433072A84BF07225A710B231B
:1082400003FB004203FB0043917A04320F2984BFF1
:108250000F2191715A7B0C330F2A84BF0F225A7061
:108260000B2202FB004302FB0042997B0C330F29D7
:1082700084BF0F21997013795279DB0343F40021F5
:1082800021611AB1254943F404230B610B2101FB41
:108290000041C979214B19B1196941F400511961A3
:1082A0000B2372B903FB0043197A9A79C90141EA99
:1082B000C221043322695B790A4342EA0312226134
:1082C0001AE003FB00431B7B144A1BB1136943F400
:1082D000805313610B2202FB0042917B557B226984
:1082E0000E4B42EAC51201F0070542EA05120907E2
:1082F00048BF42F400621A610B2202FB0040C27ABE
:10830000064B04301AB91A6981790A431A61206947
:10831000FFF710FF2369636138BD00BFA02600206E
:1083200010B5114C0023C000236123185B7F13B1EB
:108330004FF4007323612218927F0B4B1AB11A6914
:1083400042F480721A612318DA7F20440F2A84BF16
:108350000F22DA77C07F236918432061FFF7EAFE16
:108360002369236210BD00BFA026002010B5224C57
:108370004FF46023C0002361231893F82B3013B10E
:108380004FF470232361231893F8252093F82410C9
:10839000120342EA813293F826302169012B42EA26
:1083A0000102226103D1144B42F480621A61221847
:1083B00092F82710236992F8282043EA0123012A22
:1083C000236103D10C4A43F080031361221892F811
:1083D0002920094B012A03D11A6942F040021A618F
:1083E0002044236990F82A0043EA00102061FFF737
:1083F000A1FE2369E36210BDA026002038B52A4CF7
:1084000043001A18224492F9311030323F29C4BF78
:108410003F2151701A18224492F9311030323F3105
:10842000BCBFC12151701A18224492F83210303268
:108430001F2984BF1F2191704FF4402222611A1816
:10844000224492F83020012A03D1174A4FF45021D8
:10845000116104EBC00191F82B10134A51B919189E
:10846000114491F83150116905F07F0541EA052169
:1084700011610CE01D18154495F8315001F003010D
:1084800005F07C052943156945EA0125156103447A
:10849000234493F83200236918432061FFF74AFE12
:1084A0002369636338BD00BFA026002010B5830098
:1084B000244C1A18224492F83810012984BF012153
:1084C00082F838101A18224492F8391038320329E9
:1084D00084BF032151701A18224492F83A1038329E
:1084E0000F2984BF0F2191701A18224492F83B1073
:1084F0003832032984BF0321D1701A18224492F81C
:108500003C1003440F2902F1380284BF0F2111717E
:10851000234493F83C0003F1380293F8383040F4D8
:10852000202040EAC330537840EA4330937840EA51
:108530000320D37840EA43102061FFF7FBFD236955
:10854000236410BDA0260020224B012010B5032279
:108550000024052183F8300083F82900022083F8E5
:10856000264083F8274083F8284083F82A0083F8C0
:108570002B4083F8384083F8394083F83A4083F839
:108580003B4083F83C405C779C77DC7718715C71EA
:10859000DC719C711872DC721C735C7383F831108F
:1085A00083F8321083F8242083F825205A729972B8
:1085B0009A732046FFF77AFF2046FFF71FFF2046F9
:1085C000FFF7D4FE2046FFF7ABFE2046BDE8104083
:1085D000FFF712BEA0260020054B042903EBC003C1
:1085E00018BF0022D97718BF5A77FFF799BE00BF8E
:1085F000A0260020044B03EBC003597709B10422E5
:10860000DA77FFF78DBE00BFA0260020024B03EBF8
:10861000C0039977FFF784BEA0260020024B03EB2E
:10862000C000C07F704700BFA0260020024B03EBB4
:10863000C000407F704700BFA0260020024B03EB24
:10864000C000807F704700BFA0260020034B0B2294
:1086500002FB00331971FFF7CFBD00BFA026002039
:10866000034B0B2202FB00335971FFF7C5BD00BF5E
:10867000A0260020034B0B2202FB0033D971FFF729
:10868000BBBD00BFA0260020034B0B2202FB003322
:108690009971FFF7B1BD00BFA0260020034B0B224C
:1086A00002FB00331972FFF7A7BD00BFA026002010
:1086B000034B0B2202FB00335972FFF79DBD00BF35
:1086C000A0260020034B0B2202FB00339972FFF718
:1086D00093BD00BFA0260020034B0B2202FB0033FA
:1086E0001973FFF789BD00BFA0260020034B0B22A2
:1086F00002FB00335973FFF77FBD00BFA0260020A7
:10870000034B0B2202FB00339973FFF775BD00BFCB
:10871000A0260020024B0B2202FB0030007970479C
:10872000A0260020024B0B2202FB0030407970474C
:10873000A0260020024B0B2202FB0030C0797047BC
:10874000A0260020024B0B2202FB003080797047EC
:10875000A0260020024B0B2202FB0030007A70475B
:10876000A0260020024B0B2202FB0030407A70470B
:10877000A0260020024B0B2202FB0030807A7047BB
:10878000A0260020024B0B2202FB0030007B70472A
:10879000A0260020024B0B2202FB0030407B7047DA
:1087A000A0260020024B0B2202FB0030807B70478A
:1087B000A0260020034A00EB8003134483F83810FE
:1087C000FFF774BEA0260020034B00EB8002134489
:1087D0005970FFF76BBE00BFD8260020034B00EB9B
:1087E000800213449970FFF761BE00BFD8260020B5
:1087F000034B00EB80021344D970FFF757BE00BF54
:10880000D8260020034B00EB800213441971FFF7B8
:108810004DBE00BFD8260020034B00EB800018445B
:1088200090F83800704700BFA0260020024B00EBF4
:108830008000184440787047D8260020024B00EB97
:108840008000184480787047D8260020024B00EB47
:1088500080001844C0787047D8260020024B00EBF7
:108860008000184400797047D8260020034A00EBA6
:108870004003134483F83010FFF7C0BDA02600204A
:10888000034B00EB400213445970FFF7B7BD00BF24
:10889000D0260020034B00EB400213449970FFF7F1
:1088A000ADBD00BFD0260020034B00EB40001844B4
:1088B00090F83000704700BFA0260020034B00EB6B
:1088C0004000184490F90100704700BFD0260020F6
:1088D000024B00EB4000184480787047D0260020FF
:1088E000034B03EBC00383F82410FFF73FBD00BF29
:1088F000A0260020034B03EBC00383F82510FFF7ED
:1089000035BD00BFA0260020034B03EBC00383F856
:108910002610FFF72BBD00BFA0260020034B03EB62
:10892000C00383F82710FFF721BD00BFA026002059
:10893000034B03EBC00383F82810FFF717BD00BFFC
:10894000A0260020034B03EBC00383F82910FFF798
:108950000DBD00BFA0260020034B03EBC00383F82E
:108960002A10FFF703BD00BFA026002010B5064B5C
:10897000044603EBC00383F82B10FFF7F7FC2046F7
:10898000BDE81040FFF73ABDA0260020024B03EBE4
:10899000C00090F824007047A0260020024B03EB93
:1089A000C00090F825007047A0260020024B03EB82
:1089B000C00090F826007047A0260020024B03EB71
:1089C000C00090F827007047A0260020024B03EB60
:1089D000C00090F828007047A0260020024B03EB4F
:1089E000C00090F829007047A0260020024B03EB3E
:1089F000C00090F82A007047A0260020024B03EB2D
:108A0000C00090F82B007047A02600202DE9F04709
:108A1000304D1E462B1893F8443004468A46914642
:108A2000DDF82080099F042B1ED8DFE803F003083F
:108A30000D121700FFF7E0FB2B19012216E0FFF7DC
:108A400095FC2B19022211E0FFF730FD2B190322B0
:108A50000CE0FFF7D3FC2B19042207E000F0C2FF63
:108A600010B92046FFF75CFC2B19002205EBC4046B
:108A700083F8442094F82A20164B012A13D002D3FD
:108A8000022A15D021E0BAF1000F03D01B689B0C1D
:108A90008AF80030B9F1000F17D02B68C3F389238F
:108AA000A9F8003011E086B11B689B0A33600CE026
:108AB0001EB11B68DB0B5B013360B8F1000F04D003
:108AC0002B68C3F3842388F800300FB12B683B7008
:108AD000BDE8F087A026002030B9044BDA7A1AB935
:108AE0000122DA72FFF788BB704700BFA026002082
:108AF00028B9034BD97A11B1D872FFF77DBB704703
:108B0000A02600202DE9F041114AC700D31993F89F
:108B10002A600546032E904604D0032283F82A20BB
:108B2000FFF724FC2846FFF721FCD8F80040230378
:108B300044BF6FEA04346FEA1434032E05D047446F
:108B400087F82A602846FFF711FC2046BDE8F0812F
:108B5000A026002070B5084C9DF810609DF81450B8
:108B600004EBC00421766276A376E6762577BDE82D
:108B70007040FFF7D5BB00BFA026002006281AD8FA
:108B8000DFE800F004070A0D101316000A4B1B68FB
:108B900010E0094B1B6A0DE0074B5B690AE0064BCE
:108BA0001B6C07E0044B5B6B04E0034BDB6A01E0EA
:108BB000014BDB7A0B607047A02600200020704735
:108BC000034B00201870034B997AFBF71DBC00BFC4
:108BD000972D0020342D00202DE9F347924C0023DF
:108BE0002370637823B96FF00043636001236370DF
:108BF000257A8E4F4DB9E8B2FBF7B7FB78550135B2
:108C0000082DF8D1884B01221A7227250026F0B2D0
:108C1000FBF7ABFBBB5D83421BD0844B844AF05413
:108C2000B31C02EB83035B68022B05D0032B0AD035
:108C3000012B0ED168B106E058B97E4A515D012979
:108C400007D1535505E07B4B5A5D012A04BF022230
:108C50005A550136082E05F10105D8D1764F774EC9
:108C60007B7EB26813B9500702D40DE051070BD4D4
:108C7000627C5AB96C4A012151746E4AD17E012935
:108C800004D10221D17601E0002262741BB9B368DD
:108C90009A0703D40EE0B3689B070BD4A37C5BB99F
:108CA000614B01229A74634B1A7F012A04D102227C
:108CB0001A7701E00023A374FB69BBB1604D95F8FE
:108CC0000080B8F1000F11D1FFF700F95D4B5A4A4F
:108CD0001B68D269C01A80EAE073A3EBE073934289
:108CE00004D9404600F052FE01232B703B6AA3B129
:108CF000554D2F788FB9FFF7E9F8544B4E4A1B6852
:108D0000126AC01A80EAE073A3EBE073934204D9BD
:108D1000384600F03BFE01232B7022784C4D424F29
:108D200005EB4213187BDFF838E193004949DFF87F
:108D30003481002800F0FE801144009108EB02010C
:108D400001910021104673440A46FFF75FFE387810
:108D50004301EA18127B013A042A00F2D980DFE8C5
:108D600002F0033AB43AB4003B4A3C4E926812F027
:108D7000040F04EB0002D27C10D0022A03D1325C33
:108D8000002A00F0C5801D44697AFBF73DFB20787E
:108D9000FFF7AEFE23780221E21818E0012A03D182
:108DA000325C002A00F0B4802B44997AFBF72CFB4C
:108DB000207805EB4015AB7A13B9FFF78DFE03E081
:108DC000335C0BB1FFF794FE23780121E218D174D4
:108DD0000022F2549CE018F90020204F002A19DBF1
:108DE0002218D27C022A01D13A5C62B12B44597A12
:108DF000FBF70AFB2078FFF77BFE23780221E218BD
:108E0000D1740022FA542778FFF760F804EB870743
:108E1000786054E02044C37CDFF80C80012B23D120
:108E20002378FB5C9BBB4AE0E8260020F12600206B
:108E30005C2D00209E2D002008000020000801402D
:108E4000952D0020902D0020092D0020882D002038
:108E5000342D0020122D0020000C0140942D002004
:108E6000282D00202E2D0020FFF730F898F8003034
:108E70000A2108EB830205EB43139B8B52684B439B
:108E8000801A80EAE072A2EBE0729A42C8DD207894
:108E900005EB4013997AFBF7B7FA207805EB4013FE
:108EA0009B7A13B9FFF718FE03E03B5C0BB1FFF7A9
:108EB0001FFE23780121E218D1740022FA5423788E
:108EC00005EB43152B7B042B18E02218D27C9A4F1C
:108ED000022A01D13A5C62B12B44597AFBF794FA29
:108EE0002078FFF705FE23780221E218D1740022D2
:108EF000FA54237805EB43152B7B052B08D18F4BB8
:108F00009B6813F0040F4FF0080314BF73613361C3
:108F1000FEF7DCFF6369C01A80EAE073A3EBE0733D
:108F20000A2B40F38A81FBF7D9FAFEF7CFFF844B77
:108F3000586182E111440EEB0300424400F0DAFC78
:108F400000F09EFCDFF8249248BBFEF7BFFF3B78A1
:108F50000A2607EB83077A68801A5A01A918898BB9
:108F60000028B8BF4042714388420FDD7549724EF8
:108F7000C85C0F4608B9F15C41B12A441846917AA1
:108F8000FBF742FA23780022FA54F25400200090B2
:108F90000190014602460346FFF738FD4DE03B785D
:108FA000DFF8948105EB4313DB7F664EABB100F035
:108FB00067FC824600F05CFC82450ED03878335C5A
:108FC000032B02D118F8003073B305EB4013D97F9F
:108FD000FBF71AFA2378032225E000F051FC3B78D6
:108FE0000028B8BF404259F833209042F25C0DD2BD
:108FF000012A02D118F80320B2B109EBC3021846C6
:109000001179FBF701FA237801220CE0022A02D140
:1090100018F8032042B105EB43121846517AFBF7CA
:10902000F3F923780222F2542678002308F8063058
:10903000FEF74CFF04EB860670602078404E05EB8F
:1090400040139B69E3B1FBF7D5F9C8B100F018FCF8
:1090500033783D4A0028B8BF404202EB4312926980
:1090600090420DD9184600F091FC3378374A01211F
:10907000D154374A0F33D15C012904BF0221D154A6
:109080000023237600F048FC70B12D4B30491B784B
:10909000DA1C885C012804BF02208854012202FAED
:1090A00003F3227E134323762A492B4A0B783BB1E4
:1090B000207E034204D11370284B1B7803B90B7038
:1090C000137833B1227E1A409A4202D1244B0122F6
:1090D0001A7000F0D5FB20B12678224B9B5D23B996
:1090E00046E000F0C5FB0028F6D1237805EB4312DB
:1090F000D2891AB91B4AD35C002B3FD0FEF7E6FE9B
:10910000237804EB8302D26905EB4311801AC989E5
:1091100080EAE072A2EBE0720A2041438A422DDD30
:10912000114EF25C52BB1846FFF7D6FC044B0122ED
:109130001B78F25422E000BF942D0020000C014067
:10914000E8260020972D0020342D00202D2D002012
:109150009E2D0020242D00201E2D0020102D0020EB
:10916000CD2D00209C2D00209D2D0020142D0020B1
:10917000FEF7ACFE324B03EB8606F06100F080FB9D
:1091800023780028B8BF404259F833202C4F904232
:109190002C4E18460AD2FFF761FB3B7806EBC3065C
:1091A000727982420DD11846002108E0FFF756FB84
:1091B0003B7806EBC3067179884202D01846FFF768
:1091C00021FBFBF78BF9FEF781FE63691C4EC01A89
:1091D00080EAE073A3EBE0730A2B2EDD307800F019
:1091E00077FC00F04DFB28B3337805EB43156B6932
:1091F000002B1FDD00F05AFB05463078FBF736FAEE
:109200003378114A281A02EB4312526980EAE0755A
:10921000A5EBE07595420DDD184600F0B7FB3378FD
:109220000A4A0121D1540A4A1533D15C012904BFED
:109230000221D154FEF74AFE606102B0BDE8F0871A
:10924000E8260020142D0020342D00201D2D0020A4
:109250009E2D002070B5164B1A7802F0FF0112B156
:10926000012907D070BD5C680CBB9A68DB689A4224
:1092700004D11CE05C68D4B91B69C3B10D4D204614
:10928000FFF736FC697A2046FBF7BEF8E97F0A4E05
:1092900021B12046FBF7B8F8032304E00846697AB9
:1092A000FBF7B2F802233370044B00221A7070BD32
:1092B00008270020342D0020972D00209D2D002010
:1092C000B0F5803F53DBB0F1807F2ADBB0F1805FE7
:1092D00011DBB0F1804F08DB3D4B984244DC3D4B45
:1092E000021653F822301B0212E03A4B821553F853
:1092F0002230DB010CE0B0F1806F364B04DB02154D
:1093000053F822309B0103E0821453F822305B01B2
:109310005A1C90FBF3F31A445210531C90FBF2F2C8
:109320001FE0B0F5801F2B4B0CDBB0F5800F04DB8A
:10933000021453F822301B0110E0821353F822303C
:10934000DB000BE0B0F5802F04DB021353F8223072
:109350009B0003E0821253F822305B005A1C90FB02
:10936000F3F313445B1021E04FF6FF707047FF28C2
:1093700022DDB0F5805F174B0BDBB0F5804F03DBD0
:10938000021253F8223010E0821153F822305B10A1
:109390000BE0B0F5806F04DB021153F822309B1014
:1093A00003E0821053F82230DB10013303FB03F299
:1093B000824208DD581E7047002806DB054B53F833
:1093C000200000117047184670474FF0FF3070477B
:1093D0000080FE7F2CEF0008684620F007018D46D4
:1093E00031B51F4C237D032B35D8DFE803F0020293
:1093F0003030A36973B11B48012103F04DF90028F7
:10940000F9D01848A56903F0F5F8C5F10305C0B215
:1094100025442877A369124D022B0BD8AB6911485C
:109420005A1CC3F10203AA611D4495F8201003F0F1
:10943000DFF810E000220B48712103F0C1F80A4B5D
:1094400010221A6100232B7585F8243003E00023D5
:10945000237584F82430BDE831408546704700BF4D
:10946000082700200030014000080140684620F035
:1094700007018D4631B5202001F0C6FE68B3194BB7
:10948000194D1022194C1A612846002101F08FFE57
:109490002046002101F08BFE00221548032103F035
:1094A0009EF81348032103F0FDF803236B6063600B
:1094B000104B002283F824200F4A20209188C9B243
:1094C00019775188C9B259771288D2B29A7701F0C8
:1094D000A9FE4FF4007001F0A5FEBDE831408546BD
:1094E000704700BF00080140300002401C000240ED
:1094F0000030014008270020F82E0020684620F0A8
:1095000007018D4671B5012183B04FF0804003F013
:109510005FFE002800F059818D4C4FF08040012102
:1095200003F061FE237803F0FF05002B2DD1A26824
:10953000E368D31A0193A068E368C01A0028B8BF93
:109540004042FFF7BDFE0646A06A4000FFF7B8FEA6
:1095500070430090A268E3689A4207DD009AE36ACC
:109560009A42B4BF009BE36A236111E0A268E368FA
:109570009A4207DA009AE36A9A42B4BF009BE36A10
:109580005B42F1E72561656002E06FF00043019303
:10959000616822696E4B91426BD0196B9A6A0A44DA
:1095A0001A631A6B12145A63196B5A6BA1EB0242BD
:1095B0001A6359681A69914209DA5868596B1A692D
:1095C0000144914211DA5A685B6B13440EE059680A
:1095D0001A6991420BDD5868596B1A69411A914218
:1095E00003DD5A685B6BD31A00E01B696360A26BF2
:1095F000574B002A40DD1A781AB99A6B009B9A42A1
:109600003ADC2269524B3AB95868996B0028B8BFC6
:109610004042884230DA21E01A69002A11DD5A6896
:10962000002A03DD59689A6B914208DB6268484B57
:10963000002A21DA59689A6B524291421CDD9A6BDA
:109640000CE01A69002A17DA5A68002A08DA596801
:109650009A6B5242914203DD9A6B52425A600BE080
:1096600062683B4B002A07DD59689A6B914203DA26
:10967000F2E700221A635A63364B5A7E1946364B7C
:109680005B7BBAB9D80708D534488068460704D54B
:1096900060680028BCBF2E4842609D0722D52F4B32
:1096A0009B6898071ED56368002B1BDD284B0022A2
:1096B0005A6017E0DA0709D5284A926812F00402C6
:1096C00004D160680028BCBF214842609B0709D5CF
:1096D000224B9B6813F0020304D16268002AC4BFC6
:1096E0001B4A5360E26B63681344E363E36B1B1430
:1096F0002364226C019B002AB8BF5242002BB8BFE2
:109700005B429A4202DD019A114B1A64E06B226CB3
:109710000F4BA0EB0242E263E068226C0244E2607D
:1097200091F8282052B15A6C996C062A9BBF186C8C
:109730005A6C1A6C00FA02F28A1A14E05A6C062A61
:109740000ED8996C186C5A6C00FA02F20AE000BF4D
:109750000827002008000020342D002000080140C8
:109760009A6C196C0A449A6494F82420194B62BBD1
:109770001A7DCAB95A6C062A08D89A6C1649C2F3DF
:10978000090201EB8202D2F8002411E05A6C996CB4
:10979000072A124A01F00F0102EB81020CBFD2F836
:1097A0000823D2F8482303E01A7D012A04D1DA6C99
:1097B0001A620B4B10225A610122002309487121C1
:1097C00084F82420A36102F0FBFE03B0BDE87140E1
:1097D00085467047082700202CEF00082400010868
:1097E0000008014000300140024BC0001861FFF743
:1097F00031BD00BF08270020024BC0005860FFF7B2
:1098000029BD00BF082700200028B8BF4042024BF6
:10981000C0009863704700BF08270020014B986084
:10982000FFF718BD08270020014BD860FFF712BDD5
:10983000082700200028B8BF4042024B80019862F0
:10984000FFF708BD082700200028B8BF4042024BA0
:10985000C000D862FFF7FEBC08270020012802D80C
:10986000024BC0B21870FFF7F5BC00BF08270020FC
:10987000024B1869082390FBF3F07047082700207B
:10988000024B5868082390FBF3F07047082700202C
:10989000024B986B082390FBF3F0704708270020D9
:1098A000014B9868704700BF08270020014BD8681B
:1098B000704700BF08270020024B986A402390FBA6
:1098C000F3F0704708270020024BD86A082390FB6A
:1098D000F3F0704708270020014B1878704700BF4D
:1098E00008270020024B586CC0F10800C0B2704736
:1098F0000827002010B5074BDC69230910B1E40CE0
:109900006401046011B1C3F38420087002B11370C4
:1099100010BD00BF08270020034BD8689B68C31AFE
:1099200058425841704700BF082700204FF480700C
:1099300001490422FDF7A2BC302700204FF48270B9
:1099400001490422FDF79ABC342700204FF48470AB
:1099500001490422FDF792BC402700204FF480709B
:1099600001490422FDF7C6BC302700204FF4827065
:1099700001490422FDF7BEBC342700204FF4847057
:1099800001490422FDF7B6BC4027002020B9034B53
:1099900001221A7018615860704700BF0827002024
:1099A00008B588B14FF080400121002203F0F9F89A
:1099B00000200146FEF7BCFF094B0020596CBDE8B2
:1099C0000840C9B2FEF708BE0121FEF7B1FFBDE8AD
:1099D000084001214FF080400A4603F0E2B800BF82
:1099E000082700204FF08043988900F0010070475D
:1099F000082810B50CD8074CC0F108006064FFF7C8
:109A0000F1FF28B9616CBDE81040C9B2FEF7E4BDB2
:109A100010BD00BF08270020054B1A7D002AFBD18E
:109A20000122D8641A751A7D002AFCD1704700BF44
:109A30000827002030B585B0FFF790FFFFF796FFAD
:109A4000FFF79CFF0120014602F070FC4FF08040C0
:109A500002F0E2FEFAF7F7FCB0F5827F2CBF40F689
:109A6000247340F29173002501A94FF08040ADF8B6
:109A70000830ADF80450ADF80A50ADF8065002F0C9
:109A80002FFF01210A464FF0804003F08AF80121A0
:109A90004FF0804003F06BF801241C2368468DF8DA
:109AA00000308DF801408DF802408DF8034002F03F
:109AB000C5F9232368468DF800308DF801508DF8E4
:109AC00002408DF8034002F0B9F905B030BD00BF87
:109AD0002DE9F84FAD4B04465A7EAD4F4501AD4BD5
:109AE0007AB97A19127A12F0400F9A6805D09B68F9
:109AF000C2F38002C3F340091CE0C2F380099A68F4
:109B000016E07A19127A12F0400F9A6809D09B6811
:109B100082F0040283F00209C2F38002C9F3400913
:109B200008E082F004099A68C9F3800982F0020211
:109B3000C2F3400278199649037A4668485913F0EF
:109B4000400F03F03F081ABF4042C6F1000AB24678
:109B500013F0800F904B9B6814BF83F0040BC3F38A
:109B6000800B08F1FF3318BFCBF3800B072B00F2FB
:109B7000AB81DFE803F004040404BFBFBFBF874E1E
:109B8000335D013B0E2B00F29F81DFE813F00F00E5
:109B9000DC002700FC003000390040004D0071005F
:109BA000940099009D01AD0093018B01FFF78CFE9D
:109BB0003D446B7B06EB840670600120B360FFF7C9
:109BC0004DFEA8F10208B8F1010FDFF8D09194BF63
:109BD0000223042309F80430BDE8F88F002A00F0BE
:109BE0007381FFF763FE6E4B43F82400C0E0B9F1C8
:109BF000000F00F069812046FFF7C8FE062362E1EE
:109C00003D4400236B735046FFF7EEFDE8E0B9F1E9
:109C1000000F40F059814846FFF7E6FDCAF1000009
:109C2000FFF7E2FD08234EE1B9F1000F00F04C818F
:109C3000FFF73CFE80460020FFF7D6FD584B4FF063
:109C4000000953F824203D44C8EB02028AEAEA7076
:109C5000A0EBEA7085F80D9043F82420FFF7F4FD9F
:109C60004046FFF7DBFD4846FFF7F8FD09232AE1F0
:109C7000FFF752FE002800F02781FFF717FE494B3F
:109C8000A8F1030818600020FFF7AEFD0120FFF7E0
:109C9000E5FD0020FFF7C2FD0020FFF7C5FD2046CF
:109CA0000021FAF7F7FCB8F1010F00F20181012061
:109CB000FFF7D4FDAEE0B9F1000F00F00581B7E089
:109CC000B9F1000F40F00081FFF7F0FD80464846F3
:109CD000FFF78AFD3D44022098FBF0F085F80D90D7
:109CE000FFF79CFD4846BEE0FFF716FE002800F097
:109CF000EB80DDE0294E335D013B0E2B00F2E4806A
:109D0000DFE803F0081E2E3E5DE270E2E28E987DF1
:109D1000B5D8D000FFF7D8FD3D4406EB84036A7B3D
:109D2000586001209A60FFF799FDB8F1060F50D0F6
:109D3000B8F1080F4DD0194B04221A55BDE8F88F21
:109D4000B8F1060F02D13D44022304E0B8F1080F38
:109D500002D13D4400236B73FFF746FD0323B2E0BD
:109D6000A8F10503012B05D822B1B8F1060F32D1B5
:109D70000423A8E0BBF1000F00F0A6800C23A2E0B2
:109D8000B8F1050F10D13D44012312E00800002076
:109D9000342D002000080140000C01406027002005
:109DA0000C2D0020582D0020B8F1070F02D13D44A2
:109DB00000236B734042FFF717FD052383E0A8F1F2
:109DC0000503012B09D8B9F1000F06D0B8F1050F32
:109DD00001D1022377E00F2375E0BBF1000F73D0B0
:109DE000072370E0BBF1000F6ED1A8F10708B8F1AE
:109DF000010F02D93D4402236B7350460CE0BBF1C6
:109E0000000F61D1A8F10708B8F1010F02D93D4454
:109E100001236B73CAF10000FFF7E6FC0A2352E04E
:109E2000BBF1000F50D0FFF741FD06EB8403D86073
:109E30000B2348E0BBF1000F46D1FFF737FD3D444F
:109E4000804685F80DB08AEAEA70A0EBEA70FFF769
:109E5000FBFC06EB8403DB680220984498FBF0F0DF
:109E6000FFF7DCFC5846FFF7F9FC0D232BE0FFF76A
:109E700053FD48B30E233355FFF718FD134B1860FD
:109E80000020FFF7B1FC0120FFF7E8FC0020FFF7FE
:109E9000C5FC0020FFF7C8FC20460021BDE8F84FB4
:109EA000FAF7F8BB0120FFF7D9FC0020FFF79CFC74
:109EB0000E2308E006EB84039A683D4458686A73F1
:109EC000FFF7C2FC00233355BDE8F88F582D002062
:109ED000024B1A5C0AB901221A547047602700200D
:109EE000024B1A5C0AB10F221A54704760270020F7
:109EF000014B185C704700BF6027002010B5124C62
:109F00001023A360114B61609842E2600BD11033C3
:109F10000F480021236001F04AF90D48214601F065
:109F20001BF90B480AE00B4B0B480021236001F0A2
:109F30003EF90948214601F00FF907480121BDE823
:109F4000104001F034B900BF002F00200054004041
:109F50006C0002401058004044000240F7B5002653
:109F6000009601961F468388404D9BB243F4807350
:109F700083803F4B044698426960AE60EA600BD133
:109F800010333C4831462B6001F011F9394829461D
:109F900001F0E2F837480AE0374B384831462B6089
:109FA00001F005F93548294601F0D6F8334801217A
:109FB00001F0FDF8A3889BB243F48053A380A388EB
:109FC0009BB243F40063A3804FF6FF730193238891
:109FD0009BB243F480732380A38AD90706D4019AE5
:109FE000531E0193002AF7D100203CE0244A4FF68B
:109FF000FF7347F00107019317701378DBB22382D8
:10A00000A38A9A0705D4019B5A1E0192002BF7D10F
:10A01000EAE7238B9BB20093154B9C420CD14FF087
:10A02000007001F0D8F80028F9D01248002101F0A2
:10A03000BEF84FF000700BE04FF4003001F0CBF8A9
:10A040000028F9D00D48002101F0B1F84FF400309C
:10A0500001F0D0F823889BB243F400732380238857
:10A060009B05FCD4012003B0F0BD00BF002F0020F1
:10A070000054004080000240105800405800024048
:10A080002C2F002073B50025009501951E4683886E
:10A0900004469BB243F4807383804FF6FF730193B1
:10A0A000FFF72CFFA3889BB243F40063A3802388AF
:10A0B0009BB243F480732380A38AD80706D4019A05
:10A0C000531E0193002AF7D100203FE0204A4FF6AB
:10A0D000FF7306F0FE06019316701378DBB223823D
:10A0E000A38A990705D4019B5A1E0192002BF7D130
:10A0F000EAE7238B9BB20093164B9C420CD14FF4A2
:10A10000001001F068F80028F9D01348002101F090
:10A110004EF84FF400100BE04FF4005001F05BF8E4
:10A120000028F9D00D48002101F041F84FF400500B
:10A1300001F060F8A38A5A07FCD523889BB243F448
:10A140000073238023889B05FCD4012002B070BDDE
:10A150002C2F0020005400406C00024044000240BC
:10A1600010B5082086B0012102F0D4F80120014684
:10A1700002F0C4F84FF40010012102F0D7F8402398
:10A18000ADF8003003238DF8023069461C233648B1
:10A190008DF8033001F063FB802369463248ADF847
:10A1A000003001F05CFB4FF40010012102F0D6F802
:10A1B00000214FF4001002F0D1F820238DF8043074
:10A1C00006238DF8053001A801238DF806308DF89F
:10A1D000073001F033FE0023ADF808304BF6FF7373
:10A1E000ADF80A302823ADF80C304FF48063ADF899
:10A1F0000E304FF48043ADF81030FAF724F9B0F583
:10A20000827F2CBF194B1A4B02A91A48059301F003
:10A2100015FC302302A91848184CADF80C3001F099
:10A220000DFC174800F028FF1022A260154B4FF6D6
:10A23000FF72E260802221462360626100234FF4B6
:10A2400040520F4863602361A361E361236262624D
:10A25000A36200F081FF0C4800F00EFF0A4821467F
:10A2600000F07AFF06B010BD000C0140400D030065
:10A27000801A06000054004000580040002F0020C3
:10A280006C0002401054004080000240684620F0FC
:10A2900007018D4601B5002182B01C4A0191938AC5
:10A2A0009BB20193019B580506D5938A23F48063E2
:10A2B0001B041B0C93820191019B990508D5134A3D
:10A2C000938A23F480631B041B0C93820023019365
:10A2D000019BDA0508D50D4A938A23F480731B0489
:10A2E0001B0C938200230193019B1B0508D5074A91
:10A2F000938A23F400631B041B0C938200230193B5
:10A3000002B0BDE801408546704700BF00540040E0
:10A31000684620F007018D4601B5002182B01C4A35
:10A320000191938A9BB20193019B580506D5938AAC
:10A3300023F480631B041B0C93820191019B9905FC
:10A3400008D5134A938A23F480631B041B0C938261
:10A3500000230193019BDA0508D50D4A938A23F463
:10A3600080731B041B0C938200230193019B1B052C
:10A3700008D5074A938A23F400631B041B0C9382BD
:10A380000023019302B0BDE801408546704700BF3D
:10A3900000580040074B10B518681C4601460A7863
:10A3A0000B4601311AB12C2AF9D100221A7001335F
:10A3B000236010BD7027002070B5044686B02020B1
:10A3C000FDF79EF9002C03DA2D20FDF799F9644280
:10A3D00000230A2194FBF1F201FB124101AE30315E
:10A3E0001D46995514460133002AF2D1705DFDF7E0
:10A3F00087F915F1FF35F9D206B070BDFDF780B9C8
:10A400002DE9F34105460DF10700FDF793F98D4C59
:10A41000002800F0B48023799DF807008A4EE3B944
:10A420007378403398420BD1A368002B40F0A7808B
:10A4300001232371337913F0FE0F40F0A0809CE0DC
:10A440000D2801D01B2801D1002304E0A3687E2B36
:10A4500000F295800133A36091E0337913F0FE0F91
:10A4600001D1FDF74DF99DF807301F2B08D9A268DF
:10A4700074497E2A76D8501C0A448860137371E0B0
:10A48000082B06D1A368002B6CD06E4A013B936069
:10A4900068E00D2B66D1A368002B63D03379112BB4
:10A4A00012D1694B002758784030C0B2FDF728F927
:10A4B000A3689F4205D2654BD85DFDF721F90137AE
:10A4C000F6E70D20FDF71CF90023D4F80880276873
:10A4D000C4F88C301A461946424537D0012911D0AC
:10A4E00002D3022925D02FE0DFF858C10CF10C006F
:10A4F000105C202828D00CEB030181F89000013378
:10A50000012121E04F4800F10C0C12F80CC0BCF105
:10A51000200F0AD1012B04D91844002180F8901093
:10A5200001334B4F02211F440EE0184480F890C0C5
:10A5300009E0DFF810C10CF10C00105C202803D0FA
:10A540009C448CF8900001330132C5E70022C4F826
:10A550008C30234483F890200123276084F80F3146
:10A560002271A2609DF807301B2B08D10023A36045
:10A5700023713379012B02D10D20FDF7C1F894F836
:10A580000F01002600285AD02E4B83F80F61F7B236
:10A59000DFF8D880C7EBC70708EB07042C48214633
:10A5A00004F042F928B9A6796379F1072B7036D502
:10A5B00006E018F807300136002BE8D12B703DE09B
:10A5C000FFF7E8FE2B780446042B14D1214904F050
:10A5D0002BF908B900230CE020461F4904F024F9A8
:10A5E00008B9012305E01D49204604F01DF990B982
:10A5F00002236B7013E00D2B0ED1194904F014F9EE
:10A600000028E7D02046174904F00EF90028E8D0CA
:10A6100020461549E9E7204604F002F96870B207C0
:10A6200004D5FFF7B7FE04F0FBF8A870730705D553
:10A63000FFF7B0FE04F0F4F8C5F80300012002B003
:10A64000BDE8F08170270020080000207C27002052
:10A6500000280020B1040108B5040108B90401086C
:10A66000BF040108C5040108CA040108AC030108BD
:10A6700038B50B4D0446A8784030C0B2FDF740F81D
:10A6800068784030C0B2FDF73BF82078FFF794FEC1
:10A690006068FFF791FEBDE838400D20FDF730B847
:10A6A000080000207047FEE7FEE7FEE7FEE7704780
:10A6B00070477047704770477047704770477047E2
:10A6C00070477047704770477047704770477047D2
:10A6D0007047704770477047704708B5014B1B685B
:10A6E000984708BD202D002008B5024B1B689847ED
:10A6F00008BD00BF982D002008B5024B1B68984785
:10A7000008BD00BF302D002008B5024B1B689847DC
:10A7100008BD00BF542D0020704770477047704738
:10A720007047704770477047704770477047704771
:10A730007047704770477047704770477047704761
:10A740007047704770477047704770477047704751
:10A750007047704770477047704770477047704741
:10A76000704700BF08B5144B98420FD003F5A053B3
:10A77000984213D0A3F5C05398421BD14FF40070F8
:10A78000012101F0DFFD4FF400700EE04FF4806016
:10A79000012101F0D7FD4FF4806006E04FF4004046
:10A7A000012101F0CFFD4FF400400021BDE8084039
:10A7B00001F0C8BD08BD00BF0028014043680A6819
:10A7C00023F4702323F4807313430A7910B543EA0A
:10A7D000022343608A68CB6884681A43084B23408D
:10A7E00013434A7943EA420383600B7CC26A013B0C
:10A7F00022F47002DBB242EA0353C36210BD00BF11
:10A80000FDF7F1FF00230360037143718360C360B0
:10A81000012303747047836811B143F0010301E021
:10A8200023F0010383607047836811B143F48073A0
:10A8300001E023F4807383607047C9B243680AB1B2
:10A84000194301E023EA010141607047836843F046
:10A850000803836070478068C0F3C0007047836856
:10A8600043F00403836070478068C0F38000704742
:10A87000836811B143F4A00301E023F4A0038360D3
:10A8800070478068C0F3805070474368013923F4F3
:10A89000604343EA413343607047436811B143F476
:10A8A000006301E023F4006343607047092970B539
:10A8B0000DD9A1F10A0404EB44040725A540A340E7
:10A8C000C66826EA050545EA0304C4600BE001EB0F
:10A8D00041040725A54003FA04F4066926EA0505A4
:10A8E00045EA04030361062A0CD8013A02EB82020E
:10A8F0001F23934001FA02F2446B24EA03031A4334
:10A90000426370BD0C2A0CD8073A02EB82021F2367
:10A91000934001FA02F2046B24EA03031A43026330
:10A9200070BD0D3A02EB82021F23934001FA02F23E
:10A93000C46A24EA03031A43C26270BD836811B17A
:10A9400043F4801301E023F4801383607047C06CEC
:10A9500080B27047014B1868704700BF4C2401401B
:10A96000436811B143F4806301E023F480634360E2
:10A970007047436811B143F4805301E023F48053DE
:10A9800043607047836823F4E04319438160704754
:10A99000836811B143F4004301E023F40043836072
:10A9A0007047836811B143F4021301E023F40213EA
:10A9B000836070478068C0F340507047092970B5C4
:10A9C0000DD9A1F10A0404EB44040725A540A340D6
:10A9D000C66826EA050545EA0304C4600BE001EBFE
:10A9E00041040725A54003FA04F4066926EA050593
:10A9F00045EA04030361846B931CC4F301555B1B9C
:10AA0000DBB203EB83031F229A40994024EA02043D
:10AA100044EA0103836370BD836B013923F440135F
:10AA200043EA0153836370474250704728314058CE
:10AA300080B27047436823F4400323F40073194342
:10AA400041607047416282627047436823F01F0390
:10AA5000194341607047054B9A6810B142F40002F7
:10AA600001E022F400029A60704700BF0024014018
:10AA7000036819420CBF002001207047C9430160E0
:10AA800070474368006810EA112004D0C9B2194227
:10AA90000CBF0020012070476FEA11210160704750
:10AAA00008B54FF00070012101F058FCBDE80840E6
:10AAB0004FF00070002101F051BC2E4B01221A60B2
:10AAC0005A6812F0010252D00278012A1A680CBFAB
:10AAD00042F0800222F080021A604378012B254B5D
:10AAE0001A680CBF42F0400222F040021A608278DD
:10AAF000012A1A680CBF42F0200222F020021A60DC
:10AB0000C378012B1B4B1A680CBF42F0100222F0D5
:10AB100010021A600279012A1A680CBF42F008027A
:10AB200022F008021A604379012B124B1A680CBFFD
:10AB300042F0040222F004021A608279C37992077B
:10AB400042EA0362037A42EA0342437A42EA035248
:10AB50004389013B1A43074BDA611A6822F001026C
:10AB60001A60586800F0010080F00100704710463C
:10AB7000704700BF00640040037801219940354BC5
:10AB800070B5D3F8002289B242F00102C3F8002266
:10AB9000D3F81C22CC432240C3F81C228278A2B9ED
:10ABA000D3F80C2246892240C3F80C220278C588CB
:10ABB000483245EA064543F83250838802890578D1
:10ABC00043EA0242244BED005A518378012B15D100
:10ABD000204B8688D3F80C22C5880A43C3F80C2280
:10ABE000027845EA0645483243F8325043890289E3
:10ABF000057843EA0242184BED005A514378154A52
:10AC00001BB9D2F80432234002E0D2F804320B43DD
:10AC10008589C2F804320F4B2DB9D2F814522C405A
:10AC2000C2F8144206E0012D04D1D3F814220A43DD
:10AC3000C3F81422827B012A04D1D3F81C221143C9
:10AC4000C3F81C12D3F8002222F00102C3F800223C
:10AC500070BD00BF006400404466004000230370E4
:10AC600043708370C370037143718371C371032395
:10AC7000037202234372012343817047044B5A69D4
:10AC800009B1104301E022EA00005861704700BF9B
:10AC900000640040334A03469168F0B5480107D488
:10ACA0009168090106D49268D20005D40420F0BD51
:10ACB000002002E0012000E00220010101F18042B9
:10ACC00002F5C842D2F8804104F00104C2F8804184
:10ACD0001C7A5D7A3CB91E6876051E60D2F8804108
:10ACE00025432E4307E05E682C43F6005E60D2F8F1
:10ACF000807126433E43C2F880619C7A01F1804115
:10AD000004F00F049C72D2F8844101F5C84124F08C
:10AD10000F04C2F884419D7AD2F884412C43C2F8D2
:10AD200084415D7B9C7B2D0445EA0465DC7A2543E8
:10AD30001C7B45EA0425C1F8885101F5C474597C8F
:10AD40009D7C090441EA0561DD7B1B7C294341EAC6
:10AD500003236360D2F8803143F00103C2F88031ED
:10AD6000F0BD00BF0064004001281DD00FD30228B1
:10AD700029D1174A9368916803F48033926801F4EB
:10AD800000319B0B43EA1143C2F3007219E0104AF1
:10AD900091689368926801F0010103F0020343EAAD
:10ADA0008103C2F380620CE0094A9368916803F45E
:10ADB0008073926801F400719B0943EA1123C2F386
:10ADC000C062134300E00023024AD05C704700BF1A
:10ADD000006400408C040108012808D002D3022836
:10ADE0000AD07047074B9A6842F0800208E0054B92
:10ADF0009A6842F4004203E0024B9A6842F400026F
:10AE00009A60704700640040034B202208B9DA6062
:10AE100070471A61704700BF0064004010B9064BCC
:10AE2000D86803E0012804D1034B186900F003003F
:10AE300070470020704700BF00640040020102F12B
:10AE4000804303F5C84310B5D3F8B04104F00404BF
:10AE5000E4B20C7224B9D3F8B041640D0C6003E085
:10AE6000D3F8B041E4084C60D3F8B04104F00204D8
:10AE70004C72D3F8B44104F00F048C72D3F8B4319F
:10AE80001B0ACB7402F1804303F5C843D3F8B841E1
:10AE900003F5DC72CC72D3F8B841240A0C73D3F8F2
:10AEA000B841240C4C73D3F8B831BDE810401B0EE8
:10AEB0008B735368CB7353681B0A0B7453681B0C5A
:10AEC0004B7453681B0E8B74FFF79EBF044B1A68BC
:10AED00042F002021A601868C0F34000704700BFD9
:10AEE00000640040054B1A6822F002021A601868DC
:10AEF00080F00200C0F34000704700BF00640040D3
:10AF0000034B9B6918420CBF00200120704700BF13
:10AF100000640040024B9A6922EA00009861704781
:10AF200000640040202838D010D8062828D006D841
:10AF300004282FD0052848D1254B986833E00728EE
:10AF400023D0082841D1224BD86836E0B0F5007FE5
:10AF50002CD007D8402823D0B0F5807F35D11C4BAA
:10AF6000986920E0B0F5803F2AD0B0F5003F22D0AC
:10AF7000B0F5806F29D1164B9869C0F380007047F7
:10AF8000134B9868C0F300207047114B9868C0F3CA
:10AF9000004070470E4BD86814E00D4B186911E063
:10AFA0000B4B186909E000F001007047084B9869E5
:10AFB000C0F340007047064B5868C0F3001070475C
:10AFC000034B5868C0F3C00070470020704700BFB3
:10AFD00000640040202835D00CD8062824D004D89E
:10AFE000042829D005281DD07047072821D008281B
:10AFF00024D07047B0F5007F2FD005D8402823D04B
:10B00000B0F5807F24D07047B0F5803F2BD0B0F5ED
:10B01000003F2AD0B0F5806F2AD1164B9A6922F0F2
:10B0200004021EE0012201E04FF48072114B9A608D
:10B0300070474FF48032F9E7082200E010220D4BF0
:10B04000DA607047082200E010220A4B1A6170474C
:10B05000084B9A6922F0010203E0064B9A6922F03C
:10B0600002029A617047082200E01022014B5A60E8
:10B07000704700BF00640040036823F001030360D1
:10B080000023036043608360C3602D4B984234D03B
:10B0900011D83C3B98422AD006D8283B984222D06F
:10B0A0001433984221D07047264B984221D0143354
:10B0B000984220D07047244B98422DD008D8A3F551
:10B0C000677398421ED003F5627398421FD0704791
:10B0D0001E4B984229D0143398422BD0283B9842DB
:10B0E0002DD11B4B1DE01B4B12E01A4B15E0194BE9
:10B0F00017E0184B1AE0174B1DE0164B5A6842F444
:10B1000070021BE0134B5A6842F0706216E0104B5D
:10B110005A6842F00F0211E00D4B5A6842F0F002FB
:10B120000CE05A6842F4706208E0094B5A6842F435
:10B13000704203E0064B5A6842F470225A6070472E
:10B140006C000240440002401C04024044040240DF
:10B1500000040240000002408A6810B50C6A0368CF
:10B1600014430A6923F4FF4314434A6923F070032C
:10B1700014438A691443CA6914434A6A14438A6AA5
:10B18000224313430360CB6843600B6883604B68C2
:10B19000C36010BD0023036043608360C36003612C
:10B1A00043618361C36103624362836270470368E2
:10B1B00011B143F0010301E023F001030360704784
:10B1C00003680AB1194301E023EA010101607047F5
:10B1D000406880B27047C3004CBF044B044B1B68EF
:10B1E00003420CBF00200120704700BF0004024052
:10B1F00000000240C3004CBF014B024B5860704737
:10B200000004024000000240C3004CBF034B044B4B
:10B210001B6803420CBF002001207047000402405D
:10B2200000000240C3004CBF014B024B5860704706
:10B230000004024000000240044B00221A605A60E1
:10B240009A60DA60024A5A61704700BF0004014008
:10B25000FFFF0700837930B50168027943B3194BCA
:10B26000CC431D6802F1804225401D605D6802F5F7
:10B2700082322C405C6014682143116002689C6833
:10B28000D1430C409C60DC682140D9604179102991
:10B2900006D1996811439960D9680A43DA6030BDD4
:10B2A00001F1804303F5823319680A431A6030BD07
:10B2B00002F1804303F582331A6822EA0101196022
:10B2C00030BD00BF0004014000230C220360037165
:10B2D000427183717047024B1A69104318617047BD
:10B2E00000040140034B5B6918420CBF00200120A1
:10B2F000704700BF00040140014B5861704700BF18
:10B3000000040140054B1A685B69034004D01042F9
:10B310000CBF002001207047184670470004014010
:10B32000014B5861704700BF00040140044B1A688C
:10B3300002F038021A601A6810431860704700BFA4
:10B3400000200240044B1A6822F008021A601A68B2
:10B3500010431860704700BF00200240044B1A6879
:10B3600022F010021A601A6810431860704700BF7C
:10B3700000200240034B044A5A6002F188325A60AE
:10B38000704700BF0020024023016745024B1A6945
:10B3900042F080021A61704700200240014BD869D8
:10B3A0008008704700200240014B186A704700BFB8
:10B3B00000200240024BD869C0F34000704700BF34
:10B3C00000200240024B1868C0F34010704700BFD5
:10B3D00000200240044B1A6909B1104301E022EA3F
:10B3E00000001861704700BF002002400128064B92
:10B3F00003D1D86900F001007047DB6818420CBF28
:10B4000000200120704700BF00200240014BD8609F
:10B41000704700BF00200240084BDA68D10709D40A
:10B42000DA68520708D4DB6813F0100F0CBF042051
:10B43000032070470120704702207047002002401F
:10B4400013B50446FFF7E8FF01280FD164B10023CC
:10B450000193FF230193019B13B1019B013BF9E78A
:10B46000FFF7DAFF013CEFE7052002E0002C08BF00
:10B47000052002B010BD38B5054640F6FF70FFF755
:10B48000DFFF042814D10B4C40F6FF70236943F012
:10B49000020323616561236943F040032361FFF7E1
:10B4A000CFFF012804D0226941F6FD7313402361C8
:10B4B00038BD00BF0020024010B540F6FF70FFF716
:10B4C000BFFF042813D10A4C40F6FF70236943F0F4
:10B4D00004032361236943F040032361FFF7B0FFB6
:10B4E000012804D0226941F6FB731340236110BD8B
:10B4F0000020024010B540F6FF70FFF7A1FF0428BE
:10B5000029D1154C154B40F6FF70A36003F1883329
:10B51000A360236943F020032361236943F04003C0
:10B520002361FFF78DFF04280ED1226941F6DF73F6
:10B53000134023612369A52243F010032361084BC4
:10B540000F201A80FFF77CFF012804D0226941F602
:10B55000EF731340236110BD0020024023016745B3
:10B5600000F8FF1F70B505460F200E46FFF768FF75
:10B57000042817D10C4C0F20236943F001032361E9
:10B58000B3B22B80FFF75CFF042804D1360C6E8029
:10B590000F20FFF755FF012804D0226941F6FE7302
:10B5A0001340236170BD00BF0020024070B5054606
:10B5B0000F200E46FFF744FF04280FD1084C0F2040
:10B5C000236943F0010323612E80FFF739FF01282F
:10B5D00004D0226941F6FE731340236170BD00BFA1
:10B5E0000020024070B505460F200E46FFF728FFE9
:10B5F000042814D10A4C0B4B0F20A36003F18833AD
:10B60000A360236943F0100323612E80FFF718FF26
:10B61000012804D0226941F6EF731340236170BD05
:10B62000002002402301674510B504460F20FFF7B4
:10B6300007FF04283ED1204B2049E443996001F1E3
:10B64000883199601969E2B241F01001FF2A19614D
:10B6500004D1C4F30723FF2B08D10EE0184B0F20B1
:10B660001A81FFF7EDFE04281CD1F2E7144A0F20DF
:10B670005381FFF7E5FE042814D1C4F30743FF2BE1
:10B6800006D00F4A0F209381FFF7DAFE042809D174
:10B69000240EFF2C01D1042006E0094B0F20DC8191
:10B6A000FFF7CEFE012805D0034A41F6EF7311697A
:10B6B0000B40136110BD00BF00200240230167450D
:10B6C00000F8FF1F38B5054640F6FF70FFF7B8FEDB
:10B6D000042836D11B4C1C4B40F6FF70A36003F1CD
:10B6E0008833A360236943F020032361236943F077
:10B6F00040032361FFF7A4FE04281BD1226941F611
:10B70000DF7313402361236943F0100323610F4B60
:10B710000DB1002200E0A5221A8040F6FF70FFF76D
:10B720008FFE01280DD0074A41F6EF7311690B40D7
:10B73000136138BD012804D0226941F6DF7313403C
:10B74000236138BD002002402301674500F8FF1F38
:10B75000F8B5114C114B0546A36003F18833A36083
:10B760000F200E461746FFF76BFE042813D12369FE
:10B7700047F0F80743F0100323613E43084B35437D
:10B780005D800F20FFF75CFE012804D0226941F69E
:10B79000EF7313402361F8BD002002402301674589
:10B7A00000F8FF1F08B5264B98422FD011D8A3F5FB
:10B7B000006398421ED003F58063984220D0A3F521
:10B7C000006398423AD10420012100F0BBFD04201F
:10B7D0002FE01C4B98421FD003F58063984221D084
:10B7E000A3F50063984229D14020012100F0AAFD71
:10B7F00040201EE00820012100F0A4FD082018E0F0
:10B800001020012100F09EFD102012E020200121D7
:10B8100000F098FD20200CE08020012100F092FD36
:10B82000802006E04FF48070012100F08BFD4FF482
:10B8300080700021BDE8084000F084BD08BD00BF55
:10B8400000140140001C014008B50120014600F031
:10B8500079FDBDE808400120002100F073BDCB78E0
:10B86000F0B5DA0648BF8A78098803F00F0548BFAB
:10B87000154311F0FF0F1DD00468002201279740E7
:10B8800007EA0106BE4211D197004FF00F0C0CFAE7
:10B8900007FC05FA07F724EA0C04282B44EA0704FE
:10B8A00001D1466102E0482B08BF06610132082A37
:10B8B000E4D10460FF291FD94468002202F1080680
:10B8C0000127B74007EA0106BE4211D197004FF0A9
:10B8D0000F0C0CFA07FC05FA07F724EA0C04282BD6
:10B8E00044EA070401D1466102E0482B08BF066123
:10B8F0000132082AE2D14460F0BD4FF6FF730380A5
:10B90000022383700423C3707047836819420CBFFD
:10B91000002001207047806880B27047C3681942D8
:10B920000CBF002001207047C06880B270470161E1
:10B930007047416170470AB10161704741617047CA
:10B94000C160704741F480338361816183618369A1
:10B9500083697047054B1A6822F07F021204120CAB
:10B96000114341EA00101860704700BF0000014019
:10B97000014B1860704700BF1C00204230B5134ACD
:10B9800000F44015B5F5401F536884B206D15568E0
:10B9900023F0706325F0706555600FE0C20205D595
:10B9A000C0F30342032505FA02F203E0420D12013F
:10B9B00004FA02F223EA020343F0706319B1400D66
:10B9C000000184402343014A536030BD0000014020
:10B9D00001F003039B000F229A40984001F0FC0104
:10B9E00001F1804101F5803110B58C6824EA020232
:10B9F0008A608A6802438A6010BD00BF08B50E4B9A
:10BA0000984204D003F58063984208D008BD4FF4F3
:10BA10000010012100F0A2FC4FF4001006E04FF4EA
:10BA20008000012100F09AFC4FF480000021BDE865
:10BA3000084000F093BC00BF00540040F0B587B050
:10BA40000446868801A80D46314F00F015FC039886
:10BA500026F03F063604B0FBF7F7360C1FFA87FCDA
:10BA60004CEA0606A6802188EA6821F00101294BEC
:10BA70000904090C9A4221800DD85300B0FBF3F35E
:10BA80009BB20CF1010C032B1FFA8CFC98BF042312
:10BA9000A4F820C022E069884BF6FF73994205D1D3
:10BAA00002EB4202B0FBF2F39BB206E019235343D0
:10BAB000B0FBF3F39BB243F48043C3F30B020AB928
:10BAC00043F001034FF4967257434FF47A7297FB99
:10BAD000F2F70137BFB243F400432784A3832388DE
:10BAE000E9889BB243F00103238023882A8823F44A
:10BAF000816323F002031B040A431B0C13439BB214
:10BB00002380AA882B8913439BB2238107B0F0BD01
:10BB100040420F00A0860100002303808380C38081
:10BB20004FF480434BF6FF72038141F28833428029
:10BB3000C3607047038819B19BB243F0010303E06F
:10BB400023F001031B041B0C03807047838819B189
:10BB50009BB243F4006303E023F400631B041B0C5B
:10BB600083807047838819B19BB243F4805303E00C
:10BB700023F480531B041B0C83807047038819B186
:10BB80009BB243F4807303E023F480731B041B0C0B
:10BB900003807047038819B19BB243F4007303E03C
:10BBA00023F400731B041B0C03807047038819B136
:10BBB0009BB243F4806303E023F480631B041B0CFB
:10BBC00003807047838901F0FE019BB223F0FE03DE
:10BBD0000B4383817047838919B19BB243F0010302
:10BBE00003E023F001031B041B0C838170470388CF
:10BBF00019B19BB243F0400303E023F040031B0460
:10BC00001B0C0380704783889BB20AB1194301E083
:10BC100023EA01018180704701827047008AC0B227
:10BC2000704712B141F0010101E001F0FE01018213
:10BC3000704782B00190019BC85A80B202B0704731
:10BC4000038829B16FEA43436FEA53439BB201E093
:10BC5000C3F30E0303807047B1F5005F038803D17F
:10BC60009BB243F4005303E023F400531B041B0C6A
:10BC700003807047038819B19BB243F4805303E0FB
:10BC800023F480531B041B0C03807047B1F5006F35
:10BC9000038803D19BB243F4006303E023F4006301
:10BCA0001B041B0C03807047038819B19BB243F03F
:10BCB000200303E023F020031B041B0C03807047C8
:10BCC000008BC0F307207047038819B19BB243F083
:10BCD000100303E023F010031B041B0C03807047C8
:10BCE000038819B99BB243F0800303E023F080037B
:10BCF0001B041B0C03807047B1F5804F838B04D06D
:10BD000023F480431B041B0C02E09BB243F48043EA
:10BD100083837047838A008B9BB243EA004020F004
:10BD20007F407047838A008B9BB243EA004020F03B
:10BD30007F40431A584258417047838A028B9BB216
:10BD400021F07F4143EA024319420CBF0020012049
:10BD500070470B0F012B03D1C94389B28182704711
:10BD6000022B01D1838A7047062B838A05D1038871
:10BD70009BB243F0010303807047038B7047838AB3
:10BD8000028B9BB221F07F4143EA024319420CBF70
:10BD90000020012070470B0F012B03D1C94389B24A
:10BDA00081827047022B01D1838A7047062B838AD8
:10BDB00005D103889BB243F0010303807047038BD6
:10BDC000704700BF0B4B6FF070424FF0FF31C3F86C
:10BDD0008010C3F88420C3F88011C3F884210022A6
:10BDE00002F1C001013200200F2A43F82100F7D1EF
:10BDF000704700BF00E100E0094B4FF020620949A5
:10BE00005A6000229A60D9601A615A619A61DA61B7
:10BE10001A625A624FF0FF329A62DA621A6370470E
:10BE200000ED00E00000FA0540F0BF60024B40F476
:10BE30000030D860704700BF00ED00E0C27830B538
:10BE400003785AB31B4A4478D2688578D243C2F348
:10BE50000222C2F1040104FA01F10F24D4402C4063
:10BE60000C4303F00301C9002401FF228C408A40E7
:10BE700003F0FC0303F1604303F56143D3F800537F
:10BE800025EA020122400A43C3F800230378012275
:10BE9000590903F01F0302FA03F306E059090122CE
:10BEA00003F01F0302FA03F32031034A42F8213062
:10BEB00030BD00BF00ED00E000E100E000230370B2
:10BEC00043708370C3707047F8F747B9F8F747B904
:10BED000F8F747B9F8F747B90001F8F746B9F8F7A6
:10BEE00047B9024B5868C0F30930704700ED00E0D5
:10BEF00000F01F03012202FA03F34009044A403014
:10BF000052F820001840C31A58425841704700BFE9
:10BF100000E100E0014B1860704700BF00EF00E057
:10BF20004209012300F01F0003FA00F0024B6032C7
:10BF300043F82200704700BF00E100E0024B586860
:10BF4000C0F30900704700BF00ED00E000F01F03E0
:10BF5000012202FA03F34009044A803052F820001B
:10BF60001840C31A58425841704700BF00E100E032
:10BF7000014B1868704700BF00ED00E021F0604100
:10BF800021F07F01014B08439860704700ED00E00D
:10BF9000014A024BDA6070470400FA0500ED00E048
:10BFA000014A024BDA6070470100FA0500ED00E03B
:10BFB000044B1A6909B1104301E022EA000018613C
:10BFC000704700BF00ED00E0012300F01F0003FAFE
:10BFD00000F0044B5A6A09B1104301E022EA000064
:10BFE0005862704700ED00E0114B30B5DB68DB4371
:10BFF000C3F30223C3F10404A140FF2424FA03F392
:10C000001A401143C0F30122D2009440090101FA01
:10C0100002F2C0F38110800000F1604000F56D4035
:10C02000836923EA0404846185692A43826130BDFF
:10C0300000ED00E0C0F3832001238340034A506AEF
:10C040001840C31A58425841704700BF00ED00E045
:10C0500000F01F00012101FA00F0024B5A68024370
:10C060005A60704700ED00E000F01F00411E012003
:10C0700000FA01F1024B5A680A435A60704700BF48
:10C0800000ED00E0C0F3833001238340034A506A8F
:10C090001840C31A58425841704700BF00ED00E0F5
:10C0A000C0F38142094B0AB9D86A7047012A0AD104
:10C0B000C0F30152986AD300D840022A14BF00F09E
:10C0C0000F00C0B27047186B704700BF00ED00E072
:10C0D000034B10F4800F0CBF586B986B704700BF78
:10C0E00000ED00E00C4B1A6842F001021A6059683A
:10C0F0000A4A0A405A601A6822F0847222F4803296
:10C100001A601A6822F480221A605A6822F4FE0229
:10C110005A6000229A607047001002400000FFF849
:10C120000C4BB0F5803F1A6822F480321A601A680E
:10C1300022F480221A6003D0B0F5802F04D070471B
:10C140001A6842F4803202E01A6842F4A0221A60AF
:10C15000704700BF00100240034B1A6822F0F8023B
:10C1600042EAC0001860704700100240014B18609E
:10C17000704700BF00004242034B5A6822F47C1211
:10C18000114308435860704700100240014B18608B
:10C19000704700BF60004242034B5A6822F003021E
:10C1A00010435860704700BF00100240024B5868AF
:10C1B00000F00C00704700BF00100240034B5A68AB
:10C1C00022F0F00210435860704700BF0010024098
:10C1D000034B5A6822F4E06210435860704700BF76
:10C1E00000100240034B5A6822F4605242EAC00039
:10C1F0005860704700100240044B1A7809B1104390
:10C2000001E022EA00001870704700BF09100240E8
:10C21000014B1860704700BFD8004242034B5A6878
:10C2200022F4404210435860704700BF00100240A3
:10C23000064B002201281A701A7002D0042802D07E
:10C2400070471870704705221A707047201002401E
:10C25000014B1860704700BF80044242024B1A6ACB
:10C2600010431862704700BF00100240014B186075
:10C27000704700BF3C0442421C4B10B55A6802F0A4
:10C280000C02042A01D0082A01D0194A0EE05A688B
:10C290005968C2F38342CC0302F1020202D5596805
:10C2A000890301D5134900E011494A4302605968E6
:10C2B000114AC1F30311545C0168E14041605C68BC
:10C2C000C4F30224145D21FA04F484605C68C4F3AE
:10C2D000C224145DE140C1605B68C3F381331A443A
:10C2E000137CB1FBF3F1016110BD00BF00100240EF
:10C2F00000127A0000093D0094040108044B5A69B9
:10C3000009B1104301E022EA00005861704700BF04
:10C3100000100240044B9A6909B1104301E022EA7F
:10C3200000009861704700BF00100240044BDA69BA
:10C3300009B1104301E022EA0000D861704700BF54
:10C3400000100240044BDA6809B1104301E022EA10
:10C350000000D860704700BF00100240044B1A690B
:10C3600009B1104301E022EA00001861704700BFE4
:10C3700000100240014B1860704700BF4004424269
:10C38000014B1860704700BF4C004242014B1870CF
:10C39000704700BF071002404309012B074A01D133
:10C3A000136803E0022B0CBF136A536A00F01F00EE
:10C3B00023FA00F000F00100704700BF00100240B7
:10C3C00008B53120FFF7E8FF094B18705A680132B1
:10C3D0005A601A7822B95A6840F2FF139A42F0D193
:10C3E0003120FFF7D9FF003018BF012008BD00BF82
:10C3F00080280020024B5A6A42F080725A627047CD
:10C4000000100240034B9B6818420CBF0020012023
:10C41000704700BF00100240014B1870704700BF0A
:10C420000A10024008B5164B98421BD003F574431E
:10C4300098420BD0A3F5784398421FD14FF4804027
:10C440000121FFF78BFF4FF4804012E04FF4805042
:10C450000121FFF777FFBDE808404FF4805000212D
:10C46000FFF770BF4FF400400121FFF777FF4FF453
:10C4700000400021BDE80840FFF770BF08BD00BFC5
:10C48000003C00400B8810B54C88028823438C8800
:10C4900002F441522343CC8823430C8923434C8923
:10C4A00023438C892343CC89234313439BB20380CA
:10C4B000838B23F400631B041B0C83830B8A03828E
:10C4C00010BD838BF0B523F47B6323F00F031B04B3
:10C4D0001B0C8383022303840B89868B022B87B07A
:10C4E00005460C46B6B223D08B8801A8002B14BF9A
:10C4F00002270127FFF7C0FEE3882289B3F5007FFA
:10C50000019B4FF00A011CBF7F017A4301FB03F33B
:10C5100008BF1202B3FBF2F305330A229BB2B3FB4E
:10C52000F2F303F001021202C3F34F0392B200E0F0
:10C530000022991E89B2FE2928BF0022E18828BF67
:10C54000022313430B439BB22B842388628833431B
:10C5500043F400631343A2881343628913439BB2DD
:10C56000AB8307B0F0BD0023038043808380C3808A
:10C57000038143818381C3810723038270470023A2
:10C580000222038043808380C380028143817047FD
:10C59000038819B19BB243F0400303E023F040034A
:10C5A0001B041B0C03807047838B19B19BB243F4AF
:10C5B000806303E023F480631B041B0C83837047B8
:10C5C000090901238B409BB21AB1828892B21343AE
:10C5D00003E0828892B222EA030383807047838853
:10C5E0009BB20AB1194301E023EA0101818070473F
:10C5F00081817047808980B270474FF6FF6399420E
:10C60000038803D09BB243F4807303E023F4807368
:10C610001B041B0C03807047838819B19BB243F045
:10C62000040303E023F004031B041B0C8380704706
:10C63000038823F400631B041B0C038003889BB254
:10C6400019430180704703889BB243F480530380F1
:10C650007047038819B19BB243F4005303E023F4FD
:10C6600000531B041B0C03807047012914BF008B6F
:10C67000808A80B27047008A80B27047B1F5804FDF
:10C68000038803D19BB243F4804303E023F4804347
:10C690001B041B0C03807047038919420CBF002048
:10C6A00001207047202906D1038903889BB243F0FB
:10C6B000400303807047402901D0082901D1038934
:10C6C0007047C94389B20181704701F00F0201230D
:10C6D00003FA02F210B584880089A4B280B2104037
:10C6E00005D009098B401C420CBF0020012010BD61
:10C6F000552906D1038903889BB243F04003038088
:10C700007047562901D0532901D10389704701F0A0
:10C710000F01012303FA01F1C94389B20181704776
:10C72000044B04281A680CBF42F0040222F00402F1
:10C730001A60704710E000E0014B5860704700BF7E
:10C7400010E000E00128084B03D11A6842F0010212
:10C7500004E0023004D11A6822F001021A60704726
:10C7600000229A60704700BF10E000E0044B1A6896
:10C7700010B142F0020201E022F002021A6070479A
:10C7800010E000E0014B9868704700BF10E000E047
:10C79000C308022B044B0CBF1B68DB6823FA00F0B4
:10C7A00000F00100704700BF10E000E030B5048CDD
:10C7B00024F001042404240C0484058B048CADB201
:10C7C00025F0F305A4B22A4324F0020442EA03133D
:10C7D00044F001049DB221430583018430BD30B58E
:10C7E000048C24F010042404240C0484058B048C91
:10C7F00025F44075A4B22D052D0D24F0200444F03D
:10C80000100445EA022242EA033344EA01119BB2D2
:10C810008CB20383048430BD08B52E4B98423AD0C5
:10C8200010D8A3F50063984225D003F580639842A1
:10C830002BD0B0F1804F4CD101200146FFF78EFD87
:10C8400001201DE0244B984231D004D8A3F5806329
:10C85000984226D008BD214B984204D003F50063CE
:10C8600098422AD008BD4FF400600121FFF76AFD0D
:10C870004FF4006028E002200121FFF76FFD022045
:10C880000021BDE80840FFF769BD04200121FFF742
:10C8900065FD0420F4E708200121FFF75FFD082073
:10C8A000EEE710200121FFF759FD1020E8E72020D6
:10C8B0000121FFF753FD2020E2E74FF40050012152
:10C8C000FFF740FD4FF400500021BDE80840FFF79E
:10C8D00039BD08BD000C004000140040002C014090
:10C8E0000388CA8803F08F03038003889BB2134335
:10C8F0004A8813439BB203808B8883850B8803850A
:10C90000054B984203D003F50063984201D10B7A9E
:10C910000386012383827047002C0140038C70B58D
:10C9200023F001031B041B0C0384038C8488028BFB
:10C930000D8822F070021204120C4E882A430D89D1
:10C9400023F002031B043543ADB21B0C2B43CD88EF
:10C95000A4B285860D4DA84203D005F50065A84216
:10C960000FD14D8923F008032B438D8823F0040356
:10C970002B4347F6FF452540CC8989890C43A4B257
:10C980002C4384800283038470BD00BF002C0140CF
:10C99000038C30B523F010031B041B0C0384038CA1
:10C9A0008288048B0D8824F4E0442404240C23F0B2
:10C9B000200344EA05241B040D891B0C43EA0513DC
:10C9C0004D8892B243EA0513CD88A4B20587114D74
:10C9D0009BB2A84203D005F50065A84216D14D8947
:10C9E00023F080039BB243EA05134FF6BF751D4049
:10C9F0008B8845EA031347F2FF3515408A899BB2BD
:10CA000045EA8205CA8945EA820292B2828004839D
:10CA1000038430BD002C0140038C30B523F48073B7
:10CA20001B041B0C0384038C8288848B0D8824F0E8
:10CA300070042404240C23F400732C431B040D897C
:10CA40001B0C43EA05234D8892B243EA0523CD88A7
:10CA50009BB28587104DA84203D005F50065A8421A
:10CA600016D14D8923F400639BB243EA05234FF6A8
:10CA7000FF351D408B8845EA032344F6FF751540BA
:10CA80008A899BB245EA0215CA8945EA021292B226
:10CA900082808483038430BD002C0140038C30B538
:10CAA00023F480531B041B0C0384038C8488828B27
:10CAB0000D8822F4E0421204120C23F4005342EADF
:10CAC00005221B040D891B0C43EA05334D88A4B2D3
:10CAD00043EA0533CD8892B2A0F84050084D9BB28E
:10CAE000A84203D005F50065A84205D18989C4F3A1
:10CAF0000D0444EA8114A4B284808283038430BD8F
:10CB0000002C01404A880B8813438A881343CA8843
:10CB100013430A8913434A8913438A8913439BB2F7
:10CB2000A0F8443070474FF6FF73838000230380E2
:10CB3000C380438003727047002303804380838057
:10CB4000C380038143818381C38170470023012215
:10CB5000038043808280C380038170470023038069
:10CB600043808380C380038143818381704703882E
:10CB700019B19BB243F0010303E023F001039B05CD
:10CB80009B0D03807047B0F8443029B16FEA4343EE
:10CB90006FEA53439BB201E0C3F30E03A0F84430A5
:10CBA000704783899BB20AB1194301E023EA01016E
:10CBB00081817047818270470A43A0F848207047FE
:10CBC00083899BB20AB1194301E023EA0101818103
:10CBD0007047038923F007031B041B0C0381704774
:10CBE000038923F070031B041B0C19430181038983
:10CBF0009BB243F007030381704738B50D46602DA3
:10CC0000114604464FF0010202D1FFF7E8FD01E0B2
:10CC1000FFF7CCFD238923F070031B041B0C2B436F
:10CC2000238123899BB243F00703238138BD10B5CC
:10CC3000048942EA0323E4B21C43A4B221430181E4
:10CC400010BD10B50446FFF7F2FF238923F07703E8
:10CC50001B041B0C43F07703238110BD10B5044661
:10CC6000FFF7E5FF23899BB243F48043238110BD86
:10CC7000018582827047038823F070039B059B0D1A
:10CC8000194301807047038923F070031B041B0CB8
:10CC900019430181704770B50589048B068C24F413
:10CCA0004074B6B224F0030426F0220625F00705EE
:10CCB000240432432D04240C2D0C44F4807442EAE5
:10CCC0000313294344F001049EB2018104830684C6
:10CCD00070BD038B23F070031B041B0C19430183ED
:10CCE0007047038B23F4E0431B041B0C43EA012130
:10CCF0008BB203837047838B23F070031B041B0CE0
:10CD0000194381837047838B23F4E0431B041B0C7E
:10CD100043EA01218BB283837047038819B19BB228
:10CD200043F0800303E023F080039B059B0D038009
:10CD30007047838819B19BB243F0040303E023F0EA
:10CD400004031B041B0C83807047838819B19BB2BA
:10CD500043F0080303E023F008031B041B0C83804B
:10CD60007047838819B19BB243F0010303E023F0BD
:10CD700001031B041B0C83807047038B23F0080303
:10CD80001B041B0C194301837047038B23F40063BE
:10CD90001B041B0C43EA01218BB203837047838B76
:10CDA00023F008031B041B0C194381837047838BFA
:10CDB00023F400631B041B0C43EA01218BB2838321
:10CDC0007047038B23F004031B041B0C19430183DE
:10CDD0007047038B23F480631B041B0C43EA01217F
:10CDE0008BB203837047838B23F004031B041B0C5B
:10CDF000194381837047838B23F480631B041B0CCE
:10CE000043EA01218BB283837047038B23F08003B5
:10CE10001B041B0C194301837047038BC3F30E03E0
:10CE200043EA01218BB203837047838B23F0800395
:10CE30001B041B0C194381837047838BC3F30E03C0
:10CE400043EA01218BB283837047038C23F00203F2
:10CE50001B041B0C194301847047038C23F0080347
:10CE60001B041B0C194301847047038C23F020031F
:10CE70001B041B0C43EA01118BB203847047038C23
:10CE800023F080031B041B0C43EA01118BB20384C3
:10CE90007047038C23F400731B041B0C43EA01212D
:10CEA0008BB203847047038C23F400631B041B0CB8
:10CEB00043EA01218BB203847047038C23F40053AF
:10CEC0001B041B0C43EA01318BB20384704701231E
:10CED0008B408A4010B5048CA4B224EA0303038477
:10CEE000038C13439BB2038410BD04238B408A4000
:10CEF00010B5048CA4B224EA03030384038C134307
:10CF00009BB2038410BD01238B4010B5048C1830F4
:10CF1000A4B224EA0303038121F008033BB94908C2
:10CF200044584FF68F732340435043580AE0043966
:10CF3000C1F34E01445848F6FF7323404350120298
:10CF4000435892B21A43425010BD038819B19BB2A4
:10CF500043F0020303E023F002039B059B0D0380D3
:10CF60007047038819B19BB243F0040303E023F038
:10CF700004039B059B0D03807047838819B19BB206
:10CF800043F0800303E023F080031B041B0C838029
:10CF90007047038823F008039B059B0D03800388DB
:10CFA0009BB2194301807047838823F070031B04F0
:10CFB0001B0C838083889BB219438180704703894F
:10CFC00023F007031B041B0C038103899BB2194345
:10CFD00001817047038923F080031B041B0C03812C
:10CFE00003899BB219430181704781847047818511
:10CFF0007047818670470187704781877047A0F826
:10D0000040107047038B23F00C031B041B0C03839D
:10D01000038B9BB2194301837047038B23F4406356
:10D020001B041B0C0383038B9BB243EA01218BB2CD
:10D0300003837047F8B50C464988A2880029B4F8E4
:10D0400000E014BF00270227012A054614BF01266D
:10D0500002262389BEF1000F11D1FFF7A7FB284656
:10D06000E188FFF7CFFF2846394632462389FFF78C
:10D07000B6FB2846E188BDE8F840FFF7CEBFFFF7D2
:10D08000AEFB2846E188FFF7C8FF284639463246FE
:10D090002389FFF78BFB2846E188BDE8F840FFF7BE
:10D0A000B1BF838B23F00C031B041B0C8383838B86
:10D0B0009BB2194381837047838B23F440631B0425
:10D0C0001B0C8383838B9BB243EA01218BB2838346
:10D0D0007047F8B50E880D4604464988AA882B8902
:10D0E0003EB9FFF763FB2046E988BDE8F840FFF74B
:10D0F00089BF042E07D1FFF772FB2046E988BDE8FF
:10D10000F840FFF78ABF082EEF88068C1CD126F462
:10D1100080763604360C0684858B068CADB225F0FD
:10D12000F30545EA0313B6B29BB21A4326F4007323
:10D1300043EA012189B241F4807182830184394636
:10D14000BDE8F840FFF7ADBF26F480563604360C34
:10D150000684858B068C25F440752D05B6B22D0D01
:10D1600045EA022526F4005242EA013145EA03333A
:10D1700089B29BB241F48051838301843946BDE872
:10D18000F840FFF799BF0388DBB2038003889BB2A6
:10D19000194301807047808E80B27047008F80B243
:10D1A0007047808F80B27047B0F8400080B27047FF
:10D1B000808C80B27047008D80B27047038A19421C
:10D1C0000CBF002001207047C94389B2018270471B
:10D1D000038A828911EA030092B203D011420CBF84
:10D1E000002001207047C94389B20182704700BF07
:10D1F00008B5224B98422CD008D8A3F5006398427A
:10D2000017D003F5806398421BD008BD1C4B984291
:10D2100027D003F5684398422FD14FF48040012175
:10D22000FFF790F8BDE808404FF480400021FFF779
:10D2300089B84FF400300121FFF790F84FF4003027
:10D2400016E04FF480200121FFF788F84FF480208A
:10D250000EE04FF400200121FFF780F84FF400208A
:10D2600006E04FF480100121FFF778F84FF48010AA
:10D270000021BDE80840FFF771B808BD004C004030
:10D2800000500040038ACA889BB223F440531343E2
:10D2900030B503820D4682890989AB8892B20B436F
:10D2A000698922F4B0520B4322F00C0213439BB263
:10D2B0008381838AAA899BB223F4407387B0134386
:10D2C0000446838201A8FEF7D7FF049A039B0E4908
:10D2D0008C4208BF134619214B432A689200B3FBC6
:10D2E000F2F16423B1FBF3F21201100903FB1011F8
:10D2F00009013231B1FBF3F303F00F031A4392B289
:10D30000228107B030BD00BF003801404FF41653F2
:10D3100003600C2200238380C380038142818381C8
:10D3200070470B8810B54C88028A23438C88C988C3
:10D3300092B223430B4322F4706213439BB20382E5
:10D3400010BD0023038043808380C380704783899E
:10D3500019B19BB243F4005303E023F400531B04C0
:10D360001B0C83817047C1F3421310B5012401F0F7
:10D370001F01A34204FA01F101D10C3003E0022B9A
:10D380000CBF1030143003680AB1194301E023EADE
:10D390000101016010BD838A9BB20AB1194301E00B
:10D3A00023EA010181827047038A23F00F031B04E3
:10D3B0001B0C0382038A9BB2194301827047838945
:10D3C00023F400631B041B0C838183899BB21943E4
:10D3D00081817047838919B19BB243F0020303E056
:10D3E00023F002031B041B0C83817047038A23F084
:10D3F00020031B041B0C0382038A9BB21943018286
:10D400007047038A19B19BB243F4804303E023F4CD
:10D4100080431B041B0C03827047C1F30801818009
:10D4200070478088C0F30800704783899BB243F03F
:10D43000010383817047038BDBB20383038B9BB2B1
:10D4400043EA012101837047038B03F47F43038385
:10D45000038B9BB2194301837047838A19B19BB236
:10D4600043F0200303E023F020031B041B0C838202
:10D470007047838A19B19BB243F0100303E023F095
:10D4800010031B041B0C83827047838A19B19BB263
:10D4900043F0080303E023F008031B041B0C838202
:10D4A0007047838A23F004031B041B0C8382838A46
:10D4B0009BB2194381827047838A19B19BB243F0B2
:10D4C000020303E023F002031B041B0C838270475A
:10D4D000038819420CBF002001207047C94389B25C
:10D4E0000180704710B5C1F3421401F01F030122FF
:10D4F000012C02FA03F201D1838903E0022C0CBF54
:10D50000038A838A9BB21340028892B243B10123FB
:10D51000090A03FA01F111420CBF0020012010BDDD
:10D52000184610BD090A01238B40DB439BB20380E0
:10D53000704700BF684620F007018D4601B5002303
:10D540000B4A0C499818884204D20B4959589950F3
:10D550000433F5E7094B0A4A934203D2002243F809
:10D56000042BF8E701F0C4F8BDE801408546704798
:10D57000000000207C040020EC050108800400204D
:10D58000302F002081F0004102E000BF83F0004313
:10D5900030B54FEA41044FEA430594EA050F08BF4E
:10D5A00090EA020F1FBF54EA000C55EA020C7FEA12
:10D5B000645C7FEA655C00F0E2804FEA5454D4EB8F
:10D5C0005555B8BF6D420CDD2C4480EA020281EA59
:10D5D000030382EA000083EA010180EA020281EA91
:10D5E0000303362D88BF30BD11F0004F4FEA0131E3
:10D5F0004FF4801C4CEA113102D0404261EB4101F2
:10D6000013F0004F4FEA03334CEA133302D0524277
:10D6100063EB430394EA050F00F0A780A4F1010433
:10D62000D5F1200E0DDB02FA0EFC22FA05F280186D
:10D6300041F1000103FA0EF2801843FA05F3594153
:10D640000EE0A5F120050EF1200E012A03FA0EFCD2
:10D6500028BF4CF0020C43FA05F3C01851EBE371FC
:10D6600001F0004507D54FF0000EDCF1000C7EEB19
:10D6700000006EEB0101B1F5801F1BD3B1F5001F57
:10D680000CD349085FEA30004FEA3C0C04F1010476
:10D690004FEA445212F5800F80F09A80BCF1004F9F
:10D6A00008BF5FEA500C50F1000041EB045141EA21
:10D6B000050130BD5FEA4C0C404141EB010111F422
:10D6C000801FA4F10104E9D191F0000F04BF0146CD
:10D6D0000020B1FA81F308BF2033A3F10B03B3F1AB
:10D6E00020020CDA0C3208DD02F1140CC2F10C023B
:10D6F00001FA0CF021FA02F10CE002F11402D8BF99
:10D70000C2F1200C01FA02F120FA0CFCDCBF41EA64
:10D710000C019040E41AA2BF01EB0451294330BD33
:10D720006FEA04041F3C1CDA0C340EDC04F1140410
:10D73000C4F1200220FA04F001FA02F340EA0300E7
:10D7400021FA04F345EA030130BDC4F10C04C4F12D
:10D75000200220FA02F001FA04F340EA030029460D
:10D7600030BD21FA04F0294630BD94F0000F83F457
:10D77000801306BF81F480110134013D4EE77FEA3A
:10D78000645C18BF7FEA655C29D094EA050F08BF86
:10D7900090EA020F05D054EA000C04BF1946104667
:10D7A00030BD91EA030F1EBF0021002030BD5FEAAB
:10D7B000545C05D14000494128BF41F0004130BDD3
:10D7C00014F580043CBF01F5801130BD01F0004527
:10D7D00045F0FE4141F470014FF0000030BD7FEA9A
:10D7E000645C1ABF194610467FEA655C1CBF0B4695
:10D7F000024650EA013406BF52EA033591EA030FAC
:10D8000041F4002130BD00BF90F0000F04BF0021A3
:10D81000704730B54FF4806404F132044FF00005D6
:10D820004FF0000150E700BF90F0000F04BF00214F
:10D83000704730B54FF4806404F1320410F00045B5
:10D8400048BF40424FF000013EE700BF42004FEAB0
:10D85000E2014FEA31014FEA02701FBF12F07F432D
:10D8600093F07F4F81F06051704792F0000F14BF2A
:10D8700093F07F4F704730B54FF4607401F000456E
:10D8800021F0004120E700BF50EA010208BF7047C5
:10D8900030B54FF000050AE050EA010208BF7047BA
:10D8A00030B511F0004502D5404261EB41014FF423
:10D8B000806404F132045FEA915C3FF4DCAE4FF027
:10D8C00003025FEADC0C18BF03325FEADC0C18BF0E
:10D8D000033202EBDC02C2F1200300FA03FC20FA5F
:10D8E00002F001FA03FE40EA0E0021FA02F11444AC
:10D8F000C1E600BF70B54FF0FF0C4CF4E06C1CEAC1
:10D9000011541DBF1CEA135594EA0C0F95EA0C0F35
:10D9100000F0DEF82C4481EA030621EA4C5123EAA8
:10D920004C5350EA013518BF52EA033541F48011D7
:10D9300043F4801338D0A0FB02CE4FF00005E1FB8A
:10D9400002E506F00042E0FB03E54FF00006E1FBD4
:10D9500003569CF0000F18BF4EF0010EA4F1FF0417
:10D96000B6F5007F64F5407404D25FEA4E0E6D4157
:10D9700046EB060642EAC62141EA55514FEAC52068
:10D9800040EA5E504FEACE2EB4F1FD0C88BFBCF5E4
:10D99000E06F1ED8BEF1004F08BF5FEA500E50F195
:10D9A000000041EB045170BD06F0004646EA01015B
:10D9B00040EA020081EA0301B4EB5C04C2BFD4EB8D
:10D9C0000C0541EA045170BD41F480114FF0000E86
:10D9D000013C00F3AB8014F1360FDEBF002001F0F4
:10D9E000004170BDC4F10004203C35DA0C341BDC6E
:10D9F00004F11404C4F1200500FA05F320FA04F040
:10DA000001FA05F240EA020001F0004221F0004173
:10DA100010EBD37021FA04F642EB06015EEA430EE6
:10DA200008BF20EAD37070BDC4F10C04C4F1200516
:10DA300000FA04F320FA05F001FA04F240EA0200C9
:10DA400001F0004110EBD37041F100015EEA430E9A
:10DA500008BF20EAD37070BDC4F1200500FA05F2BA
:10DA60004EEA020E20FA04F301FA05F243EA020339
:10DA700021FA04F001F0004121FA04F220EA020048
:10DA800000EBD3705EEA430E08BF20EAD37070BD8E
:10DA900094F0000F0FD101F00046400041EB01016E
:10DAA00011F4801F08BF013CF7D041EA060195F050
:10DAB000000F18BF704703F00046520043EB03030A
:10DAC00013F4801F08BF013DF7D043EA06037047F7
:10DAD00094EA0C0F0CEA135518BF95EA0C0F0CD002
:10DAE00050EA410618BF52EA4306D1D181EA030148
:10DAF00001F000414FF0000070BD50EA410606BF42
:10DB00001046194652EA430619D094EA0C0F02D186
:10DB100050EA013613D195EA0C0F05D152EA0336CB
:10DB20001CBF104619460AD181EA030101F00041E9
:10DB300041F0FE4141F470014FF0000070BD41F032
:10DB4000FE4141F4780170BD70B54FF0FF0C4CF40C
:10DB5000E06C1CEA11541DBF1CEA135594EA0C0F2B
:10DB600095EA0C0F00F0A7F8A4EB050481EA030E78
:10DB700052EA03354FEA013100F088804FEA03335F
:10DB80004FF0805545EA131343EA12634FEA02222D
:10DB900045EA111545EA10654FEA00260EF00041EE
:10DBA0009D4208BF964244F1FD0404F5407402D240
:10DBB0005B084FEA3202B61A65EB03055B084FEAD1
:10DBC00032024FF480104FF4002CB6EB020E75EBCE
:10DBD000030E22BFB61A754640EA0C005B084FEAF6
:10DBE0003202B6EB020E75EB030E22BFB61A754673
:10DBF00040EA5C005B084FEA3202B6EB020E75EBBE
:10DC0000030E22BFB61A754640EA9C005B084FEA35
:10DC10003202B6EB020E75EB030E22BFB61A754642
:10DC200040EADC0055EA060E18D04FEA051545EA31
:10DC300016754FEA06164FEAC30343EA52734FEADA
:10DC4000C2025FEA1C1CC0D111F4801F0BD141EA53
:10DC500000014FF000004FF0004CB6E711F4801FB8
:10DC600004BF01430020B4F1FD0C88BFBCF5E06F98
:10DC70003FF6AFAEB5EB030C04BFB6EB020C5FEAA8
:10DC8000500C50F1000041EB045170BD0EF0004EFD
:10DC90004EEA113114EB5C04C2BFD4EB0C0541EA2F
:10DCA000045170BD41F480114FF0000E013C90E62C
:10DCB00045EA060E8DE60CEA135594EA0C0F08BFF0
:10DCC00095EA0C0F3FF43BAF94EA0C0F0AD150EAEF
:10DCD00001347FF434AF95EA0C0F7FF425AF104682
:10DCE00019462CE795EA0C0F06D152EA03353FF4AA
:10DCF000FDAE1046194622E750EA410618BF52EA27
:10DD000043067FF4C5AE50EA41047FF40DAF52EAFA
:10DD100043057FF4EBAE12E74FF0FF3C06E000BF97
:10DD20004FF0010C02E000BF4FF0010C4DF804CDA4
:10DD30004FEA410C7FEA6C5C4FEA430C18BF7FEA64
:10DD40006C5C1BD001B050EA410C0CBF52EA430C92
:10DD500091EA030F02BF90EA020F0020704710F112
:10DD6000000F91EA030F58BF994208BF90422CBFA1
:10DD7000D8176FEAE37040F0010070474FEA410C9A
:10DD80007FEA6C5C02D150EA013C07D14FEA430CB8
:10DD90007FEA6C5CD6D152EA033CD3D05DF8040B29
:10DDA000704700BF8446104662468C46194663465B
:10DDB00000E000BF01B5FFF7B7FF002848BF10F132
:10DDC000000F01BD4DF808EDFFF7F4FF0CBF012077
:10DDD00000205DF808FB00BF4DF808EDFFF7EAFFF3
:10DDE00034BF012000205DF808FB00BF4DF808EDAE
:10DDF000FFF7E0FF94BF012000205DF808FB00BFA3
:10DE00004DF808EDFFF7CEFF94BF012000205DF82C
:10DE100008FB00BF4DF808EDFFF7C4FF34BF012039
:10DE200000205DF808FB00BF4FEA4102B2F1E04379
:10DE300024BFB3F5001CDCF1FE5C0DD901F0004CF1
:10DE40004FEAC0024CEA5070B2F1004F40EB830041
:10DE500008BF20F00100704711F0804F21D113F16D
:10DE60003872BCBF01F00040704741F480114FEAA6
:10DE70005252C2F11802C2F1200C10FA0CF320FA2F
:10DE800002F018BF40F001004FEAC1234FEAD3234C
:10DE900003FA0CFC40EA0C0023FA02F34FEA4303B6
:10DEA000CCE77FEA625307D150EA01331EBF4FF03F
:10DEB000FE4040F44000704701F0004040F0FE405A
:10DEC00040F40000704700BF80F0004002E000BF57
:10DED00081F0004142001FBF5FEA410392EA030F55
:10DEE0007FEA226C7FEA236C6AD04FEA1262D2EB9F
:10DEF0001363C1BFD218414048404140B8BF5B42A4
:10DF0000192B88BF704710F0004F40F4000020F03C
:10DF10007F4018BF404211F0004F41F4000121F052
:10DF20007F4118BF494292EA030F3FD0A2F101029C
:10DF300041FA03FC10EB0C00C3F1200301FA03F1DA
:10DF400000F0004302D5494260EB4000B0F5000FFD
:10DF500013D3B0F1807F06D340084FEA310102F1BC
:10DF60000102FE2A51D2B1F1004F40EBC25008BF6E
:10DF700020F0010040EA03007047490040EB000038
:10DF800010F4000FA2F10102EDD1B0FA80FCACF167
:10DF9000080CB2EB0C0200FA0CF0AABF00EBC25066
:10DFA00052421843BCBFD0401843704792F0000F54
:10DFB00081F4000106BF80F400000132013BB5E7A7
:10DFC0004FEA41037FEA226C18BF7FEA236C21D01D
:10DFD00092EA030F04D092F0000F08BF0846704782
:10DFE00090EA010F1CBF0020704712F07F4F04D150
:10DFF000400028BF40F00040704712F100723CBF63
:10E0000000F50000704700F0004343F0FE4040F48C
:10E01000000070477FEA226216BF08467FEA23634A
:10E020000146420206BF5FEA412390EA010F40F435
:10E03000800070474FF0000304E000BF10F0004381
:10E0400048BF40425FEA000C08BF704743F0964368
:10E0500001464FF000001CE050EA010208BF704783
:10E060004FF000030AE000BF50EA010208BF70470A
:10E0700011F0004302D5404261EB41015FEA010C1F
:10E0800002BF84460146002043F0B64308BFA3F117
:10E090008053A3F50003BCFA8CF2083AA3EBC253F9
:10E0A00010DB01FA02FC634400FA02FCC2F1200218
:10E0B000BCF1004F20FA02F243EB020008BF20F04F
:10E0C0000100704702F1200201FA02FCC2F12002B5
:10E0D00050EA4C0021FA02F243EB020008BF20EAAA
:10E0E000DC70704742000ED2B2F1FE4F0BD34FF0FE
:10E0F0009E03B3EB126209D44FEA002343F00043BE
:10E1000023FA02F070474FF00000704712F1610FE0
:10E1100001D1420202D14FF0FF3070474FF00000B2
:10E12000704700BF73B96AB9002908BF0028BCBF97
:10E1300000204FF00041C4BF6FF000414FF0FF30AE
:10E1400000F03CB882B0EC462DE9005000F006F833
:10E15000DDF804E002B00CBC704700BF2DE9704F41
:10E16000089E14461D468046894600F029F804FBA7
:10E1700001F3A4FB00AB00FB05329344B8EB0A08A3
:10E1800069EB0B09C6E90089BDE8708F2DE9704F76
:10E19000089E14461D468046894600F061F900FB42
:10E1A00005F5A0FB04AB04FB0154A344B8EB0A083B
:10E1B00069EB0B09C6E90089BDE8708F704700BFA5
:10E1C00000292DE9F00FC0F2A1800024002BC0F23D
:10E1D0009880154606460F46002B3FD18A4258D9F3
:10E1E000B2FA82F34BB1C3F1200201FA03F720FA2D
:10E1F00002F29D4000FA03F61743290CB7FBF1F237
:10E2000001FB1277A8B200FB02F34FEA164C4CEA6E
:10E210000747BB4209D97F1902F1FF3C80F0058115
:10E22000BB4240F20281023A2F44FF1AB7FBF1F3DE
:10E2300001FB137100FB03F0B6B246EA01418842CC
:10E2400008D9491903F1FF3780F0F180884240F284
:10E25000EE80023B43EA0242002303E08B420AD9EC
:10E2600000231A461046194614B1404261EB4101A1
:10E27000BDE8F00F7047B3FA83F8B8F1000F40F033
:10E2800088808B4202D3824200F2E2800023012286
:10E29000E8E712B90123B3FBF2F5B5FA85F2002ADB
:10E2A0003AD17F1B280C1FFA85FC0123B7FBF0F144
:10E2B00000FB11770CFB01F24FEA164848EA0747CA
:10E2C000BA4207D97F1901F1FF3802D2BA4200F2EF
:10E2D000C4804146BF1AB7FBF0F200FB12700CFB82
:10E2E00002FCB6B246EA0040844507D9401902F163
:10E2F000FF3702D2844500F2AE803A4642EA01423C
:10E30000B0E7E443524263EB430362E7404261EB10
:10E3100041014FF0FF3459E79540C2F1200927FA37
:10E3200009F126FA09F99740280CB1FBF0F800FB37
:10E3300018111FFA85FC0CFB08F349EA07094FEA9C
:10E34000194747EA01418B4206FA02F608D94919F2
:10E3500008F1FF327AD28B4278D9A8F10208294419
:10E36000C91AB1FBF0F300FB13170CFB03F21FFA01
:10E3700089F949EA0747BA4207D97F1903F1FF3102
:10E3800060D2BA425ED9023B2F44BF1A43EA084327
:10E390008CE7C8F1200225FA02F103FA08FC27FAFB
:10E3A00002F320FA02F207FA08F741EA0C0C4FEAEE
:10E3B0001C49B3FBF9F109FB11331FFA8CFA0AFB74
:10E3C00001FB17433A0C42EA03439B4505FA08F068
:10E3D00008D913EB0C0301F1FF3235D29B4533D939
:10E3E00002396344CBEB0303B3FBF9F209FB1233AD
:10E3F0000AFB02FABFB247EA0347BA4508D917EB4E
:10E400000C0702F1FF331BD2BA4519D9023A67440F
:10E4100042EA0145A5FB0001CAEB07078F424FF016
:10E4200000030AD305D02A461CE76246FDE63B46B8
:10E4300010E706FA08F68642F5D26A1E002311E7B5
:10E440001A46E5E70B46A0E71146CBE7904687E77B
:10E450004346424606E7023A50E702392F4439E77D
:10E460002DE9F00F144605460E46002B43D18A4293
:10E4700053D9B2FA82F757B1C7F1200620FA06F64F
:10E4800001FA07F302FA07F400FA07F51E43210C1C
:10E49000B6FBF1F201FB1266A0B200FB02F32F0CF7
:10E4A00047EA0646B34209D9361902F1FF3780F030
:10E4B000FD80B34240F2FA80023A2644F61AB6FBD7
:10E4C000F1F301FB136100FB03F0ADB245EA01413A
:10E4D000884208D9091903F1FF3680F0E9808842A3
:10E4E00040F2E680023B43EA02420023104619460E
:10E4F000BDE8F00F70478B424CD8B3FA83F6002E7C
:10E500004FD18B4202D3824200F2DD80BDE8F00F92
:10E510000023012210461946704712B90124B4FBAA
:10E52000F2F4B4FA84F2002A40F08280091B260C2F
:10E53000A7B20123B1FBF6F006FB101107FB00F2B6
:10E540004FEA154C4CEA01418A4207D9091900F1FA
:10E55000FF3C02D28A4200F2C8806046891AB1FBB1
:10E56000F6F206FB121107FB02F7ADB245EA0145D0
:10E57000AF4208D92C1902F1FF3180F09B80A742ED
:10E5800040F29880023A42EA004210461946BDE83D
:10E59000F00F704700231A4610461946BDE8F00FE9
:10E5A0007047C6F1200522FA05F703FA06F421FAAE
:10E5B00005F301FA06FB20FA05F53C434FEA14483F
:10E5C000B3FBF8FC08FB1C331FFA84F909FB0CFAB7
:10E5D00045EA0B0B4FEA1B4545EA03439A4502FA0D
:10E5E00006F204D91B190CF1FF356FD3AC46CAEB08
:10E5F0000303B3FBF8F508FB153309FB05F91FFA14
:10E600008BFB4BEA0347B94504D93F1905F1FF33AA
:10E6100062D31D4645EA0C4CACFB0223C9EB07074D
:10E620009F424FF000054AD346D062462B465DE735
:10E630009440C2F1200921FA09FC914020FA09F91D
:10E64000260CBCFBF6F806FB18CCA7B207FB08F3B8
:10E6500049EA01094FEA194141EA0C4C634500FAC5
:10E6600002F509D91CEB040C08F1FF323BD26345DB
:10E6700039D9A8F10208A444C3EB0C0CBCFBF6F397
:10E6800006FB13C107FB03F21FFA89F949EA0141AE
:10E690008A4207D9091903F1FF3022D28A4220D9D0
:10E6A000023B2144891A43EA084343E73A4605E717
:10E6B000334618E70A4666E7B0409042B5D20CF1FF
:10E6C000FF32002312E7334632460FE79A458DD9D1
:10E6D000ACF1020C23448AE7B9459AD9023D27449C
:10E6E00098E70346DEE79046C6E70238214435E75F
:10E6F00070B5414EFDF7F6FC00254FF480303570C3
:10E70000FDF70EFDFDF75CFE0128044621D1102027
:10E71000FCF724FE2046FCF709FE4FF48030294622
:10E72000FDF72AFD2046FDF731FD3920FDF734FEC7
:10E730000028FAD00220FDF72FFDFDF737FD08284D
:10E74000FBD10020FDF73AFD0020FDF74BFD012332
:10E75000337001200146FDF7DDFD4FF0C05001216F
:10E76000FDF7E4FD4FF480414FF00060FDF706FC3B
:10E77000224D4FF44070FDF757FBF5F701FDF6F71A
:10E7800027F800232B701E4A1E4B1F4C1A601F4A8D
:10E790001F4B1A601F4B204A1A60F5F73FFEFBF72C
:10E7A000DFFCF9F799FBF9F773FBF8F735FEF5F79E
:10E7B0008DFD2078F8F78AFEE078F8F7D3FF2B7804
:10E7C00023B96079A1682269F9F706F9F9F7BCFE67
:10E7D000F5F7A4FFFBF72EF9F8F70AF9F9F778FC3B
:10E7E000FAF7EEF90D4B08225A61F8F7EBF9FAF750
:10E7F000F3F9F9F76EFCF8E78C2D0020082D0020C6
:10E8000019790008202D002008000020B9770008A1
:10E81000982D0020302D0020697800080008014064
:10E8200000210A2200F0ACB80F4B30B405461C683A
:10E8300002E0D01A16D1ABB115F8013BE2185078BE
:10E840001A4600F00300012808BF03F1200211F866
:10E85000013BE018407800F003000128E9D12033A3
:10E86000D01AE9D030BC7047740400202DE9F00FB5
:10E87000424C82B0D4F800C001900E4600E026461B
:10E88000344614F8015B0CEB0500407800F00800FA
:10E8900000F0FF0A0028F2D12D2D5BD02B2D04BFF4
:10E8A0007578B41C33F010003CD09946BAF1000FD3
:10E8B0000CBF6FF0004B4FF0004BBBFBF9F800278B
:10E8C00009FB18BB38460CE0303DAB4219DD7E1C1D
:10E8D00005D0404523D820D009FB0050012714F86B
:10E8E000015B0CEB0506767816F0040FECD116F000
:10E8F000030606D0012E14BF57263726AD1BAB42A8
:10E90000E5DC7B1C15D0BAF1000F21D10AB1EFB9BB
:10E91000116002B0BDE8F00F70475D45DCDD4FF0DF
:10E92000FF37DCE7302D1AD0002BBED10A239946E1
:10E93000BCE70199BAF1000F4FF022030CBF6FF052
:10E9400000404FF000400B60002AE2D0611EDFE77C
:10E950004042DBE7B41C75784FF0010AA2E720784B
:10E9600000F0DF00582803D0002B9ED108239CE73D
:10E97000102365789946023498E700BF740400209C
:10E9800030B4044C0D46134601462A46206830BC7C
:10E99000FFF76CBF700400202DE9F0418AB00446F7
:10E9A0000D4600F06DF8DFF8D080064698F900308B
:10E9B0000F4601330BD02046294600F059FA30B1FA
:10E9C0002046294600220023FFF724FA20B13046D2
:10E9D00039460AB0BDE8F081234B98F800600890F2
:10E9E000CDE90245CDE90445019346BB1F4B4FF0ED
:10E9F0006042CDE906232046294600220023FFF786
:10EA0000E1F970B102239E42009322D0684600F0E3
:10EA100057FAF0B1089B0BBBDDE906010AB0BDE86F
:10EA2000F0810123022E00930ED0684600F048FAD0
:10EA300050B10F4800F046FACDE90601EAE70D4B68
:10EA40000022CDE90623D6E700F042FA2123036035
:10EA5000EFE700F03DFA22230360DBE700F038FA2D
:10EA6000089B0360D8E700BFDC050108FFFFEFC784
:10EA7000E00501080000F0FF78040020000000001D
:10EA80002DE9F04FB1F5801F87B002460B460F46C7
:10EA90005BDA21F00046064300F0F5800029C0F261
:10EAA000A4810022B24BFEF725FF0F460B46B14969
:10EAB00002468F426FF035054BDCC7F3130606F5AF
:10EAC000152101F6647101F4801484F07F5181F402
:10EAD000401141EA0603104619460022A64BFEF7F4
:10EAE00055FD4FEA2758B31CA8F2FF38C3F31303B0
:10EAF000A844022B08EB145882468B464FF00002C4
:10EB00002EDC0023FFF75EF9002800F0C580B8F185
:10EB1000000F00F071814046FEF786FE80A3D3E926
:10EB2000002306460F46FEF7E5FE7FA3D3E9002348
:10EB300004460D4630463946FEF7DCFE02460B46DB
:10EB400020462946FEF724FD07E08A4900258F422A
:10EB5000B3DD10461946FEF71BFD07B0BDE8F08F88
:10EB60004FF08043FEF714FD02460B4650465946CF
:10EB7000FEF7EAFFCDE902014046FEF755FECDE97A
:10EB80000401DDE9020102460B46FEF7B3FE024630
:10EB90000B46CDE90001FEF7ADFE65A3D3E90023E6
:10EBA00004460D46FEF7A6FE63A3D3E90023FEF755
:10EBB000EFFC22462B46FEF79DFE61A3D3E900231E
:10EBC000FEF7E6FC22462B46FEF794FE5EA3D3E951
:10EBD0000023FEF7DDFCDDE90023FEF78BFE5CA3DE
:10EBE000D3E90023CDE9000120462946FEF782FE45
:10EBF00059A3D3E90023FEF7CBFC22462B46FEF7B0
:10EC000079FE57A3D3E90023FEF7C2FC22462B4628
:10EC1000FEF770FE0B460246DDE90001FEF7B8FC88
:10EC2000A6F5C223C6F5D726A3F27A4351361E4372
:10EC3000002E04460D4657DD0022504B50465946E3
:10EC4000FEF758FE52465B46FEF754FE06460F4658
:10EC5000B8F1000F40F0968022462B46FEF798FC54
:10EC6000DDE90223FEF746FE02460B4630463946F2
:10EC7000FEF78CFC02460B4650465946FEF786FCD2
:10EC800007B0BDE8F08F0022002300203C49FEF7CA
:10EC90005BFF07B0BDE8F08F52465B4650465946D1
:10ECA000FEF728FE30A3D3E9002304460D46504664
:10ECB0005946FEF71FFE02460B4600202F49FEF77D
:10ECC00065FC02460B4620462946FEF713FE044625
:10ECD0000D46B8F1000F40F092805046594622464A
:10ECE0002B46FEF753FC38E7B8F1000F00F0AB807D
:10ECF0000BA3D3E90023DDE90401FEF7FBFD224667
:10ED00002B4606460F4650465946FEF73FFCDDE9C6
:10ED10000223FEF7EFFD04460D46DDE904017CE029
:10ED20000000E0FE422EE63F763C7935EF39EA3DC1
:10ED300044523EDF12F1C23FDE03CB966446C73F2A
:10ED4000599322942449D23F935555555555E53F43
:10ED50009FC678D0099AC33FAF788E1DC571CC3F4E
:10ED600004FA97999999D93F555555555555D53F19
:10ED700000005043FFFFEF7F0000F03F0000E03F46
:10ED8000000050C336A3D3E90023DDE90401FEF7F8
:10ED9000B1FD2246804689462B4630463946FEF76D
:10EDA000F7FBDDE90223FEF7A5FD2FA3D3E900233E
:10EDB00004460D46DDE90401FEF79CFD02460B46C4
:10EDC00020462946FEF7E4FB02460B46304639460C
:10EDD000FEF7DCFB52465B46FEF7D8FB02460B46CD
:10EDE00040464946FEF7D2FBB7E6FEF7CFFB0022CE
:10EDF0000023FEF7A9FEB0E600200021ADE6404664
:10EE0000FEF712FD16A3D3E9002380468946FEF7DC
:10EE100071FD06460F464046494613A3D3E9002339
:10EE2000FEF768FD02460B4620462946FEF7AEFB7C
:10EE300052465B46FEF7AAFB02460B463046394671
:10EE4000FEF7A4FB89E602460B4650465946FEF7FC
:10EE50009DFBDDE90223FEF74DFD0BE7AFF30080DC
:10EE60000000E0FE422EE63F763C7935EF39EA3D80
:10EE700031F0004310B408D00F4AA3F58014944237
:10EE80000AD804205DF8044B704700280CBF02200C
:10EE900003205DF8044B7047B3F5801F01D20320B7
:10EEA000F7E7064A934201D00020F2E7D0F10100D3
:10EEB00038BF0020EDE700BFFFFFDF7F0000F07FDD
:10EEC0000020704700200149704700BF0000F87F14
:10EED000014B1868704700BF7004002050C3000049
:10EEE0008813000001800808000000000064000092
:10EEF0000000000000000000C800000000D4300046
:10EF0000801A060000000000000000000000000061
:10EF100000000000000000000000000000000000F1
:10EF200000000000000000000000000000000000E1
:10EF300010000000160000001B0000002000000070
:10EF400023000000270000002A0000002D00000020
:10EF500030000000320000003500000037000000E3
:10EF6000390000003B0000003D00000040000000B0
:10EF70004100000043000000450000004700000081
:10EF8000490000004B0000004C0000004E00000053
:10EF90005000000051000000530000005400000029
:10EFA0005600000057000000590000005A00000001
:10EFB0005B0000005D0000005E00000060000000DB
:10EFC00061000000620000006300000065000000B6
:10EFD0006600000067000000680000006A00000092
:10EFE0006B0000006C0000006D0000006E0000006F
:10EFF000700000007100000072000000730000004B
:10F00000740000007500000076000000770000002A
:10F0100078000000790000007A0000007B0000000A
:10F020007C0000007D0000007E00000080000000E9
:10F0300080000000810000008200000083000000CA
:10F0400084000000850000008600000087000000AA
:10F0500088000000890000008A0000008B0000008A
:10F060008C0000008D0000008E0000008F0000006A
:10F07000900000009000000091000000920000004D
:10F08000930000009400000095000000960000002E
:10F090009600000097000000980000009900000012
:10F0A0009A0000009B0000009B0000009C000000F4
:10F0B0009D0000009E0000009F000000A0000000D6
:10F0C000A0000000A1000000A2000000A3000000BA
:10F0D000A3000000A4000000A5000000A60000009E
:10F0E000A7000000A7000000A8000000A900000081
:10F0F000AA000000AA000000AB000000AC00000065
:10F10000AD000000AD000000AE000000AF00000048
:10F11000B0000000B0000000B1000000B20000002C
:10F12000B2000000B3000000B4000000B500000011
:10F13000B5000000B6000000B7000000B7000000F6
:10F14000B8000000B9000000B9000000BA000000DB
:10F15000BB000000BB000000BC000000BD000000C0
:10F16000BD000000BE000000BF000000C0000000A5
:10F17000C0000000C1000000C1000000C20000008B
:10F18000C3000000C3000000C4000000C500000070
:10F19000C5000000C6000000C7000000C700000056
:10F1A000C8000000C9000000C9000000CA0000003B
:10F1B000CB000000CB000000CC000000CC00000021
:10F1C000CD000000CE000000CE000000CF00000007
:10F1D000D0000000D0000000D1000000D1000000ED
:10F1E000D2000000D3000000D3000000D4000000D3
:10F1F000D4000000D5000000D6000000D6000000BA
:10F20000D7000000D7000000D8000000D90000009F
:10F21000D9000000DA000000DA000000DB00000086
:10F22000DB000000DC000000DD000000DD0000006D
:10F23000DE000000DE000000DF000000E000000053
:10F24000E0000000E1000000E1000000E20000003A
:10F25000E2000000E3000000E3000000E400000022
:10F26000E5000000E5000000E6000000E600000008
:10F27000E7000000E7000000E8000000E8000000F0
:10F28000E9000000EA000000EA000000EB000000D6
:10F29000EB000000EC000000EC000000ED000000BE
:10F2A000ED000000EE000000EE000000EF000000A6
:10F2B000F0000000F0000000F1000000F10000008C
:10F2C000F2000000F2000000F3000000F300000074
:10F2D000F4000000F4000000F5000000F50000005C
:10F2E000F6000000F6000000F7000000F700000044
:10F2F000F8000000F8000000F9000000F90000002C
:10F30000FA000000FA000000FB000000FB00000013
:10F31000FC000000FC000000FD000000FD000000FB
:10F32000FE000000FE000000FF00000001F00100F0
:10F3300002F0010004F0010005F0010007F00100F7
:10F3400008F001000AF001000BF001000DF00100CF
:10F350000EF0010010EE010011EE010013EE0100AD
:10F3600015EE010016EE010018EE010019EE010085
:10F370001BEE01001CEC01001EEC01001FEC010063
:10F3800021EC010022EC010024EA010025EA010041
:10F3900027EA010028EA01002AE801002BE8010021
:10F3A0002DE801002EE8010030E6010031E6010001
:10F3B00033E6010034E4010036E4010037E40100E3
:10F3C00039E201003AE201003CE201003DE00100C7
:10F3D0003EE0010040E0010041DE010043DE0100AB
:10F3E00044DC010046DC010047DC010049DA010091
:10F3F0004ADA01004CD801004DD801004FD6010077
:10F4000050D6010051D4010053D4010054D2010060
:10F4100056D2010057D0010059D001005ACE010048
:10F420005BCE01005DCC01005ECA010060CA010034
:10F4300061C8010062C8010064C6010065C4010022
:10F4400067C4010068C2010069C201006BC001000D
:10F450006CBE01006DBE01006FBC010070BA0100FE
:10F4600072B8010073B8010074B6010076B40100EF
:10F4700077B4010078B201007AB001007BAE0100E0
:10F480007CAE01007EAC01007FAA010080A80100D3
:10F4900081A8010083A6010084A4010085A20100C7
:10F4A00087A00100889E0100899E01008A9C0100BE
:10F4B0008C9A01008D9801008E9601008F940100B6
:10F4C000919201009292010093900100948E0100AC
:10F4D000968C0100978A01009888010099860100A6
:10F4E0009A8401009C8201009D8001009E7E0100A3
:10F4F0009F7C0100A07A0100A1780100A3760100A1
:10F50000A4740100A5720100A6700100A76E01009D
:10F51000A86C0100A96A0100AA680100AC6601009C
:10F52000AD640100AE620100AF600100B05E010099
:10F53000B15C0100B25A0100B3580100B45401009B
:10F54000B5520100B6500100B74E0100B84C0100A1
:10F55000B94A0100BA480100BB460100BC420100A3
:10F56000BD400100BE3E0100BF3C0100C03A0100A9
:10F57000C1380100C2340100C3320100C4300100AF
:10F58000C52E0100C62C0100C7280100C8260100B5
:10F59000C9240100C9220100CA1E0100CB1C0100C0
:10F5A000CC1A0100CD180100CE140100CF120100C9
:10F5B000CF100100D00E0100D10A0100D2080100D5
:10F5C000D3060100D4020100D4000100D5FE0000E2
:10F5D000D6FC0000D7F80000D7F60000D8F40000F1
:10F5E000D9F00000DAEE0000DAEC0000DBE8000001
:10F5F000DCE60000DCE40000DDE00000DEDE000010
:10F60000DFDA0000DFD80000E0D60000E1D2000021
:10F61000E1D00000E2CE0000E2CA0000E3C8000032
:10F62000E4C40000E4C20000E5C00000E5BC000046
:10F63000E6BA0000E7B60000E7B40000E8B2000058
:10F64000E8AE0000E9AC0000E9A80000EAA600006E
:10F65000EAA20000EBA00000EB9E0000EC9A000084
:10F66000EC980000ED940000ED920000EE8E00009A
:10F67000EE8C0000EE880000EF860000EF820000B4
:10F68000F0800000F07C0000F07A0000F1780000CB
:10F69000F1740000F1720000F26E0000F26C0000E4
:10F6A000F2680000F3660000F3620000F3600000FF
:10F6B000F45C0000F45A0000F4560000F45400001A
:10F6C000F5500000F54E0000F54A0000F548000036
:10F6D000F6440000F6420000F63E0000F63C000052
:10F6E000F6380000F7360000F7320000F73000006F
:10F6F000F72C0000F72A0000F7260000F722000090
:10F70000F7200000F81C0000F81A0000F8160000AE
:10F71000F8140000F8100000F80E0000F80A0000CD
:10F72000F8080000F8040000F8020000F8020200E7
:10F73000F8040200F8080200F80A0200F80E0200BD
:10F74000F8100200F8140200F8160200F81A02007D
:10F75000F81C0200F7200200F7220200F726020040
:10F76000F72A0200F72C0200F7300200F7320200FD
:10F77000F7360200F6380200F63C0200F63E0200C0
:10F78000F6420200F6440200F5480200F54A020083
:10F79000F54E0200F5500200F4540200F456020047
:10F7A000F45A0200F45C0200F3600200F36202000B
:10F7B000F3660200F2680200F26C0200F26E0200D0
:10F7C000F1720200F1740200F1780200F07A020096
:10F7D000F07C0200F0800200EF820200EF8602005F
:10F7E000EE880200EE8C0200EE8E0200ED92020026
:10F7F000ED940200EC980200EC9A0200EB9E0200ED
:10F80000EBA00200EAA20200EAA60200E9A80200B8
:10F81000E9AC0200E8AE0200E8B20200E7B4020080
:10F82000E7B60200E6BA0200E5BC0200E5C002004D
:10F83000E4C20200E4C40200E3C80200E2CA02001B
:10F84000E2CE0200E1D00200E1D20200E0D60200E6
:10F85000DFD80200DFDA0200DEDE0200DDE00200B7
:10F86000DCE40200DCE60200DBE80200DAEC020085
:10F87000DAEE0200D9F00200D8F40200D7F6020056
:10F88000D7F80200D6FC0200D5FE0200D400030027
:10F89000D4020300D3060300D2080300D10A0300F8
:10F8A000D00E0300CF100300CF120300CE140300CC
:10F8B000CD180300CC1A0300CB1C0300CA1E0300A2
:10F8C000C9220300C9240300C8260300C728030077
:10F8D000C62C0300C52E0300C4300300C33203004E
:10F8E000C2340300C1380300C03A0300BF3C030028
:10F8F000BE3E0300BD400300BC420300BB46030004
:10F90000BA480300B94A0300B84C0300B74E0300DD
:10F91000B6500300B5520300B4540300B3580300BB
:10F92000B25A0300B15C0300B05E0300AF60030095
:10F93000AE620300AD640300AC660300AA68030076
:10F94000A96A0300A86C0300A76E0300A670030059
:10F95000A5720300A4740300A3760300A17803003A
:10F96000A07A03009F7C03009E7E03009D8003001D
:10F970009C8203009A840300998603009888030000
:10F98000978A0300968C0300948E030093900300E3
:10F9900092920300919203008F9403008E960300CD
:10F9A0008D9803008C9A03008A9C0300899E0300B3
:10F9B000889E030087A0030085A2030084A403009F
:10F9C00083A6030081A8030080A803007FAA030088
:10F9D0007EAC03007CAE03007BAE03007AB0030074
:10F9E00078B2030077B4030076B4030074B6030062
:10F9F00073B8030072B8030070BA03006FBC030051
:10FA00006DBE03006CBE03006BC0030069C203003F
:10FA100068C2030067C4030065C4030064C6030032
:10FA200062C8030061C8030060CA03005ECA030025
:10FA30005DCC03005BCE03005ACE030059D0030017
:10FA400057D0030056D2030054D2030053D403000E
:10FA500051D4030050D603004FD603004DD8030005
:10FA60004CD803004ADA030049DA030047DC0300FC
:10FA700046DC030044DC030043DE030041DE0300F8
:10FA800040E003003EE003003DE003003CE20300F1
:10FA90003AE2030039E2030037E4030036E40300EE
:10FAA00034E4030033E6030031E6030030E60300EC
:10FAB0002EE803002DE803002BE803002AE80300EA
:10FAC00028EA030027EA030025EA030024EA0300EA
:10FAD00022EC030021EC03001FEC03001EEC0300EA
:10FAE0001CEC03001BEE030019EE030018EE0300EC
:10FAF00016EE030015EE030013EE030011EE0300F3
:10FB000010EE03000EF003000DF003000BF00300F5
:10FB10000AF0030008F0030007F0030005F00300FB
:10FB200004F0030002F0030001F0030001F1030000
:10FB300002F1030004F1030005F1030007F10300E3
:10FB400008F103000AF103000BF103000DF10300BB
:10FB50000EF1030010EF030011EF030013EF030099
:10FB600015EF030016EF030018EF030019EF030071
:10FB70001BEF03001CED03001EED03001FED03004F
:10FB800021ED030022ED030024EB030025EB03002D
:10FB900027EB030028EB03002AE903002BE903000D
:10FBA0002DE903002EE9030030E7030031E70300ED
:10FBB00033E7030034E5030036E5030037E50300CF
:10FBC00039E303003AE303003CE303003DE10300B3
:10FBD0003EE1030040E1030041DF030043DF030097
:10FBE00044DD030046DD030047DD030049DB03007D
:10FBF0004ADB03004CD903004DD903004FD7030063
:10FC000050D7030051D5030053D5030054D303004C
:10FC100056D3030057D1030059D103005ACF030034
:10FC20005BCF03005DCD03005ECB030060CB030020
:10FC300061C9030062C9030064C7030065C503000E
:10FC400067C5030068C3030069C303006BC10300F9
:10FC50006CBF03006DBF03006FBD030070BB0300EA
:10FC600072B9030073B9030074B7030076B50300DB
:10FC700077B5030078B303007AB103007BAF0300CC
:10FC80007CAF03007EAD03007FAB030080A90300BF
:10FC900081A9030083A7030084A5030085A30300B3
:10FCA00087A10300889F0300899F03008A9D0300AA
:10FCB0008C9B03008D9903008E9703008F950300A2
:10FCC000919303009293030093910300948F030098
:10FCD000968D0300978B0300988903009987030092
:10FCE0009A8503009C8303009D8103009E7F03008F
:10FCF0009F7D0300A07B0300A1790300A37703008D
:10FD0000A4750300A5730300A6710300A76F030089
:10FD1000A86D0300A96B0300AA690300AC67030088
:10FD2000AD650300AE630300AF610300B05F030085
:10FD3000B15D0300B25B0300B3590300B455030087
:10FD4000B5530300B6510300B74F0300B84D03008D
:10FD5000B94B0300BA490300BB470300BC4303008F
:10FD6000BD410300BE3F0300BF3D0300C03B030095
:10FD7000C1390300C2350300C3330300C43103009B
:10FD8000C52F0300C62D0300C7290300C8270300A1
:10FD9000C9250300C9230300CA1F0300CB1D0300AC
:10FDA000CC1B0300CD190300CE150300CF130300B5
:10FDB000CF110300D00F0300D10B0300D2090300C1
:10FDC000D3070300D4030300D4010300D5FF0200CE
:10FDD000D6FD0200D7F90200D7F70200D8F50200DD
:10FDE000D9F10200DAEF0200DAED0200DBE90200ED
:10FDF000DCE70200DCE50200DDE10200DEDF0200FC
:10FE0000DFDB0200DFD90200E0D70200E1D302000D
:10FE1000E1D10200E2CF0200E2CB0200E3C902001E
:10FE2000E4C50200E4C30200E5C10200E5BD020032
:10FE3000E6BB0200E7B70200E7B50200E8B3020044
:10FE4000E8AF0200E9AD0200E9A90200EAA702005A
:10FE5000EAA30200EBA10200EB9F0200EC9B020070
:10FE6000EC990200ED950200ED930200EE8F020086
:10FE7000EE8D0200EE890200EF870200EF830200A0
:10FE8000F0810200F07D0200F07B0200F1790200B7
:10FE9000F1750200F1730200F26F0200F26D0200D0
:10FEA000F2690200F3670200F3630200F3610200EB
:10FEB000F45D0200F45B0200F4570200F455020006
:10FEC000F5510200F54F0200F54B0200F549020022
:10FED000F6450200F6430200F63F0200F63D02003E
:10FEE000F6390200F7370200F7330200F73102005B
:10FEF000F72D0200F72B0200F7270200F72302007C
:10FF0000F7210200F81D0200F81B0200F81702009A
:10FF1000F8150200F8110200F80F0200F80B0200B9
:10FF2000F8090200F8050200F8030200F8030000D7
:10FF3000F8050000F8090000F80B0000F80F0000B9
:10FF4000F8110000F8150000F8170000F81B000079
:10FF5000F81D0000F7210000F7230000F72700003C
:10FF6000F72B0000F72D0000F7310000F7330000F9
:10FF7000F7370000F6390000F63D0000F63F0000BC
:10FF8000F6430000F6450000F5490000F54B00007F
:10FF9000F54F0000F5510000F4550000F457000043
:10FFA000F45B0000F45D0000F3610000F363000007
:10FFB000F3670000F2690000F26D0000F26F0000CC
:10FFC000F1730000F1750000F1790000F07B000092
:10FFD000F07D0000F0810000EF830000EF8700005B
:10FFE000EE890000EE8D0000EE8F0000ED93000022
:10FFF000ED950000EC990000EC9B0000EB9F0000E9
:020000040801F1
:10000000EBA10000EAA30000EAA70000E9A90000B4
:10001000E9AD0000E8AF0000E8B30000E7B500007C
:10002000E7B70000E6BB0000E5BD0000E5C1000049
:10003000E4C30000E4C50000E3C90000E2CB000017
:10004000E2CF0000E1D10000E1D30000E0D70000E2
:10005000DFD90000DFDB0000DEDF0000DDE10000B3
:10006000DCE50000DCE70000DBE90000DAED000081
:10007000DAEF0000D9F10000D8F50000D7F7000052
:10008000D7F90000D6FD0000D5FF0000D401010023
:10009000D4030100D3070100D2090100D10B0100F4
:1000A000D00F0100CF110100CF130100CE150100C8
:1000B000CD190100CC1B0100CB1D0100CA1F01009E
:1000C000C9230100C9250100C8270100C729010073
:1000D000C62D0100C52F0100C4310100C33301004A
:1000E000C2350100C1390100C03B0100BF3D010024
:1000F000BE3F0100BD410100BC430100BB47010000
:10010000BA490100B94B0100B84D0100B74F0100D9
:10011000B6510100B5530100B4550100B3590100B7
:10012000B25B0100B15D0100B05F0100AF61010091
:10013000AE630100AD650100AC670100AA69010072
:10014000A96B0100A86D0100A76F0100A671010055
:10015000A5730100A4750100A3770100A179010036
:10016000A07B01009F7D01009E7F01009D81010019
:100170009C8301009A8501009987010098890100FC
:10018000978B0100968D0100948F010093910100DF
:1001900092930100919301008F9501008E970100C9
:1001A0008D9901008C9B01008A9D0100899F0100AF
:1001B000889F010087A1010085A3010084A501009B
:1001C00083A7010081A9010080A901007FAB010084
:1001D0007EAD01007CAF01007BAF01007AB1010070
:1001E00078B3010077B5010076B5010074B701005E
:1001F00073B9010072B9010070BB01006FBD01004D
:100200006DBF01006CBF01006BC1010069C301003B
:1002100068C3010067C5010065C5010064C701002E
:1002200062C9010061C9010060CB01005ECB010021
:100230005DCD01005BCF01005ACF010059D1010013
:1002400057D1010056D3010054D3010053D501000A
:1002500051D5010050D701004FD701004DD9010001
:100260004CD901004ADB010049DB010047DD0100F8
:1002700046DD010044DD010043DF010041DF0100F4
:1002800040E101003EE101003DE101003CE30100ED
:100290003AE3010039E3010037E5010036E50100EA
:1002A00034E5010033E7010031E7010030E70100E8
:1002B0002EE901002DE901002BE901002AE90100E6
:1002C00028EB010027EB010025EB010024EB0100E6
:1002D00022ED010021ED01001FED01001EED0100E6
:1002E0001CED01001BEF010019EF010018EF0100E8
:1002F00016EF010015EF010013EF010011EF0100EF
:1003000010EF01000EF101000DF101000BF10100F1
:100310000AF1010008F1010007F1010005F10100F7
:1003200004F1010002F1010001F10100E0C002004E
:1003300060C0030060C10300E0C10200E0C1000032
:1003400060C1010060C00100E0C00000E0C0020028
:1003500060C0030060C10300E0C10200E0C1000012
:1003600060C1010060C00100E0C00000B46901008C
:10037000B4680100B4680300B4690300B469010003
:10038000B4680100B4680300B4690300B4690100F3
:10039000B4680100B4680300B4690300B4690100E3
:1003A000B4680100B4680300B4690300524F5200FE
:1003B000000106524F4C000002064D53540000034A
:1003C000024D5650000004075341500000050747F6
:1003D000415000000603535441500007035253415B
:1003E00050000803534750000009074747500000DA
:1003F0000A0353544750000B0352534750000C0359
:1004000052465300000D0353494F00000E07474961
:100410004F00000F0353414300001D0753434F009B
:10042000001E0747434F00001F0343434F000020B7
:100430000341434F00002703554630000040075555
:100440004631000041075546320000420755463309
:100450000000430755463400004407554635000068
:100460004507554636000046075546370000470702
:1004700052554E0000810553544F500080004249B0
:100480004E00008B00000000000000000200000091
:100490000000000100000000010203040102030447
:1004A0000607080902040608313032315631343269
:1004B000004142530052454C00434F4F52440053B9
:1004C000544152540053544F5000535441545553C7
:1004D00000000000430000000020202020202020F9
:1004E00020202828282828202020202020202020E4
:1004F00020202020202020202088101010101010F4
:10050000101010101010101010040404040404043F
:1005100004040410101010101010414141414141D9
:1005200001010101010101010101010101010101BB
:1005300001010101101010101010424242424242CB
:10054000020202020202020202020202020202028B
:100550000202020210101010200000000000000033
:10056000000000000000000000000000000000008B
:10057000000000000000000000000000000000007B
:10058000000000000000000000000000000000006B
:10059000000000000000000000000000000000005B
:1005A000000000000000000000000000000000004B
:1005B000000000000000000000000000000000003B
:1005C000000000000000000000000000000000002B
:1005D0000000000000000000000000006C6F6700D9
:0405E0000000000017
:0805E400DCDBFF7F01000000D9
:1005EC00A80401080001000000010200000800003E
:1005FC0001000000020000000000000000000000EC
:10060C0000000000000000000000000000000000DE
:10061C0000000000000000000000000000000000CE
:10062C000000000000000000000000003403002067
:10063C009C030020040400200000000000000000C7
:10064C00000000000000000000000000000000009E
:10065C00000000000000000000000000D4040108AD
:10066C00000000000000000000000000000000007E
:10067C00000000000000000000000000000000006E
:10068C00000000000000000000000000000000005E
:10069C00000000000000000000000000000000004E
:1006AC00000000000000000000000000000000003E
:1006BC00000000000000000000000000000000002E
:1006CC00000000000000000000000000000000001E
:1006DC0001000000000000000E33CDAB34126DE6BB
:1006EC00ECDE05000B000000000000000000000024
:1006FC0000000000000000000000000000000000EE
:10070C0000000000000000000000000000000000DD
:10071C0000000000000000000000000000000000CD
:10072C0000000000000000000000000000000000BD
:0C0A5C0048000020D80401080100000040
:04000005080041109E
:00000001FF
